:10632800E5467006127B928F4622E546B4050612B2
:106338003B738F4622E546B40B0612719E8F4622A8
:10634800E546B40A061268838F4622E546B40F066E
:10635800126C8E8F4622E546B414061265348F46B9
:1063680022E546B41906127AD58F4622E546B41EB0
:1063780006127BA68F4622E546B42306126CE48FEC
:106388004622E546B42806127C5B8F4622E546B4D1
:106398002D06127BBA8F4622E546B4320512743FA9
:0363A8008F4622FB
:107B9200C20890061EE0FFA3E0901CECCFF0A3EF1A
:047BA200F07F052249
:103B7300127C5750477D047F011262A05008E53E36
:103B8300B401037F0B227D047F021262A05008E57B
:103B93003EB402037F0B227D047F031262A0500810
:103BA300E53EB403037F0B227D047F041262A05021
:103BB30008E53EB404037F0B227F0A227F081276B6
:103BC30023500612546D7F00227D057F051262A0EB
:103BD3005032901CEEE07002A3E070282046257D51
:103BE300017F011262A04003023CE990066CE0FFF2
:103BF3007C0A7D70127384900610E0FFA3E0901C92
:103C0300EE023CB07D067F051262A05031901CF09D
:103C1300E07002A3E070272048247D017F02126236
:103C2300A04003023CE990066DE0FF7C0A7D901200
:103C33007384900612E0FFA3E0901CF0806F7D0771
:103C43007F051262A05031901CF2E07002A3E07075
:103C530027204C247D017F031262A04003023CE92C
:103C630090066EE0FF7C0A7DB0127384900614E028
:103C7300FFA3E0901CF280357D087F051262A050FF
:103C830033901CF4E07002A3E07029204F267D01DD
:103C93007F041262A0504F90066FE0FF7C0A7DD034
:103CA300127384900616E0FFA3E0901CF4CFF0A3F8
:103CB300EFF080327D077F061262A0500F30290C8F
:103CC300901CECE07002A3E07002C22930380C9023
:103CD3001CECE07002A3E07002C238786CE6B40515
:093CE300057F04125DEC7F05224F
:10719E00203842900633E0901D10F0123346E53E43
:1071AE00B401062049247F0522E53EB40206204D97
:1071BE00197F0522E53EB4030620510E7F0522E518
:1071CE003EB404062054037F0522901D10E0D39494
:0871DE000050C8D2387F0A22DC
:10688300E53B700AE53EB40105753B018028E53B15
:10689300700AE53EB40205753B02801AE53B700AB7
:1068A300E53EB40305753B03800CE53B7008E53E0C
:1068B300B40403753B047D077F061262A0500C7D70
:1068C300077F061262A0501E30291B900650E0FF7E
:1068D3007C067DF01273847D017F011262A0500655
:0968E300120FB3122B647F0F2287
:106C8E00127C57503F120FB3202F092030062031AF
:106C9E0003303209E53270051277E7800B786CE627
:106CAE00B4050B7F03125DEC122B64120FB3202F71
:106CBE001020300D20310A203207E5327003122BDE
:106CCE00647F0F221277E77D057F071262A05003C3
:066CDE007F14227F00225A
:10653400E4F53B7D077F061262A0500C7D077F06C1
:106544001262A0505E30295B786CE670047F018093
:1065540008786CE6B404077F02125DEC8038786C2E
:10656400E6B407047601802E7D037F051262A050F5
:1065740025901CF6E07002A3E0701B900662E0FF19
:106584007C097D30127384900620E0FFA3E0901C08
:10659400F6CFF0A3EFF07F0612762350037F00229C
:1065A4007F19227D077F061262A050052029027FF1
:0265B4000522BE
:107AD5007D077F061262A050062029037F052290AC
:0A7AE5000630E0901D10F07F1E2215
:107BA600901D10E070037F2322127C5750037F0A3A
:047BB600227F1E22EA
:106CE4007D047F071262A05041E53EB4010B90067B
:106CF4005EE0FF7C087DB0802EE53EB4020B90067A
:106D04005FE0FF7C087DD0801EE53EB4030B900657
:106D140060E0FF7C087DF0800EE53EB4040C900634
:106D240061E0FF7C097D10127384900631E0901DB0
:056D340010F07F282291
:037C5B007F2D2258
:107BBA00901D10E070037F3222127C5750037F0A17
:047BCA00227F2D22C7
:10743F003058037F32227D047F051262A0502890BE
:10744F001CF8E07002A3E0701E900663E0FF7C0959
:10745F007D50127384900622E0FFA3E0901CF8CFBA
:0C746F00F0A3EFF07F3222C2087F002261
:10730100900640E06035D259D224753D03123346D0
:10731100122B64120FB3127C575009E53D60051220
:10732100334680F2E4F522F523127C574009E53D0E
:10733100600512334680F2E53D70D2C259C224C2C3
:027341005822D0
:04000E0001000630B7
:030003000269B4DB
:0B69B400C0E0C083C082C0D075D008D6
:1069BF00853082852F83E493FF204404C4540FFF56
:1069CF00430FF08F80C284D28500C2870000D28728
:1069DF00007580FF7580FEC284C28500C2870000EB
:1069EF000000D287007580FF30440CC2440530E5AB
:0B69FF00307006052F8002D244D2A8A1
:096A0A00D0D0D082D083D0E0325C
:03000B00021BB61F
:101BB600C0E0C0F0C083C082C0D075D008758CD894
:101BC600758A92D28C12433B127588E531D3940004
:101BD60040051531021F40753111901D10E0D39458
:101BE600004003E014F0901D11E0D394004003E0A0
:101BF60014F0901D12E0D394004003E014F0901D01
:101C060013E0D394004003E014F0E532D39400408F
:101C16000215321541E541B40A004003021F3D900A
:101C26001C2CF8282873021F40021E91021E59021E
:101C36001E2C021DC2021D58021CEE021C84021C30
:101C460067021C4AD3901CEDE09400901CECE094D3
:101C5600005003021F40A3E024FFF0901CEC021F7B
:101C660031D3901CE9E09400901CE8E09400500306
:101C7600021F40A3E024FFF0901CE8021F317F0101
:101C86001278AF4003021F40901CE1E09400901CC4
:101C9600E0E09400400CA3E024FFF0901CE0E03468
:101CA600FFF0D3901CEFE09400901CEEE09400400F
:101CB6000CA3E024FFF0901CEEE034FFF0D3901C60
:101CC600FBE09400901CFAE094005003021F407D54
:101CD600067F011262A04003021F40901CFBE02415
:101CE600FFF0901CFA021F317F021278AF40030208
:101CF6001F40901CE3E09400901CE2E09400400C2E
:101D0600A3E024FFF0901CE2E034FFF0D3901CF136
:101D1600E09400901CF0E09400400CA3E024FFF057
:101D2600901CF0E034FFF0D3901CFDE09400901C72
:101D3600FCE094005003021F407D067F021262A061
:101D46004003021F40901CFDE024FFF0901CFC02A3
:101D56001F317F031278AF4003021F40901CE5E05D
:101D66009400901CE4E09400400CA3E024FFF09063
:101D76001CE4E034FFF0D3901CF3E09400901CF2D6
:101D8600E09400400CA3E024FFF0901CF2E034FF46
:101D9600F0D3901CFFE09400901CFEE094005003EA
:101DA600021F407D067F031262A04003021F40907F
:101DB6001CFFE024FFF0901CFE021F317F04127806
:101DC600AF4003021F40901CE7E09400901CE6E041
:101DD6009400400CA3E024FFF0901CE6E034FFF0F2
:101DE600D3901CF5E09400901CF4E09400400CA302
:101DF600E024FFF0901CF4E034FFF0D3901D01E0E6
:101E06009400901D00E094005003021F407D067F61
:101E1600041262A04003021F40901D01E024FFF05F
:101E2600901D00021F31D3901CEBE09400901CEA39
:101E3600E09400400CA3E024FFF0901CEAE034FF9D
:101E4600F0901D14E0D394005003021F40E014F0FC
:101E5600021F40D3901CF9E09400901CF8E0940017
:101E6600400CA3E024FFF0901CF8E034FFF0D39080
:101E76001CF7E09400901CF6E094005003021F400B
:101E8600A3E024FFF0901CF6021F31786CE6FF7089
:101E960003021F40EFB401059006188027786CE610
:101EA600FFB40219D3901CEBE09400901CEAE09476
:101EB60000403FA3E024FFF0901CEA806EEFB403DD
:101EC6001190061AE0FFA3E0901CEACFF0A3EFF012
:101ED6008020786CE6FFB4041ED3901CEBE09400DF
:101EE600901CEAE09400400AA3E024FFF0901CEA6C
:101EF6008039786C068043EF6405603E786CE6FFB7
:101F0600B4060D901CEA7402F0A37458F006802AF9
:101F1600EFB40726D3901CEBE09400901CEAE09403
:101F260000400EA3E024FFF0901CEAE034FFF080AE
:101F360009786C7600800375410A127A824008128D
:101F460076B54003127A9ED0D0D082D083D0F0D01E
:021F5600E03277
:03001300026188FF
:0D618800C0E0C0F0C083C082C0D075D01050
:1061950075A0FFC284C285D287C286308018C2A48A
:1061A500C2A5D2A6C2A7E5A0540FF54AD2A7FF12F1
:1061B5006636D286804F308118D2A4C2A5D2A6C237
:1061C500A7E5A0540FF54AD2A7FF1263ABD286808C
:1061D50034308218C2A4D2A5D2A6C2A7E5A0540F16
:1061E500F54AD2A7FF12642ED2868019308316D2C3
:1061F500A4D2A5D2A6C2A7E5A0540FF54AD2A7FFFF
:056205001264B1D28615
:0B620A00D0D0D082D083D0F0D0E032A2
:106C3700BF0113900632E0901D10F0901D10E0D3B5
:106C47009400404280F5BF0213900632E0901D1178
:106C5700F0901D11E0D39400402C80F5BF031390F2
:106C67000632E0901D12F0901D12E0D394004016FA
:106C770080F5BF0411900632E0901D13F0901D13AC
:076C8700E0D3940050F72256
:106D3900304712205F0F900672E0FF7C0B7D301206
:106D49007384D25F22304B1220610F900673E0FFEB
:106D59007C0B7D50127384D26122304E1220620F57
:106D6900900674E0FF7C0B7D70127384D26222302E
:106D7900521120630E900675E0FF7C0B7D90127313
:046D890084D263222B
:10561800303D1A204617900664E0FF7C097D701221
:105628007384D246C214C210C21CC2182230461457
:10563800203911900665E0FF7C097D90127384C2C1
:1056480046C23D22303E1A204817900666E0FF7C8D
:10565800097DB0127384D248C215C211C21DC21985
:1056680022304814203A11900667E0FF7C097DD06B
:10567800127384C248C23E2230401A204C1790064A
:1056880068E0FF7C097DF0127384D24CC216C21206
:10569800C21EC21A22304C14203B11900669E0FF4A
:1056A8007C0A7D10127384C24CC2402230421A20F8
:1056B8004F1790066AE0FF7C0A7D30127384D24F40
:1056C800C217C213C21FC21B22304F13203C1090B6
:1056D800066BE0FF7C0A7D50127384C24FC24222DF
:1052A200124221D28C7F07127623500512001680FB
:1052B2001212722E7F1F7E001278D690001FEFF01E
:1052C20012770F7F0812762350051259E180FE9063
:1052D20006087402F0A37458F090060A7402F0A350
:1052E2007458F090060C7402F0A37458F090060EF5
:1052F2007402F0A37458F0900681E0FF7C0D7D10DB
:10530200127384E4FFEFFD3395E0FC74302DF582D7
:1053120074003CF583E0FE74F02DF582741A3CF5BE
:1053220083EEF00FBF08DED208127A9E7545017F28
:1053320001125DEC900618E0FFA3E0901CEACFF0AA
:10534200A3EFF0C208127A9E123346305A11E53E9C
:10535200B4010C900651E0FF7C077D101273841299
:105362006328305B03124566305C03124453305DA0
:10537200031249A9306003124AB3124FC27D077F5C
:10538200061262A04002C229125618126D3980B864
:104566007C007D80C2677F011236B950117F06122A
:1045760076235002D2087F01121F580246067C009D
:104586007D70D2677F011236B95002800D7C007DA6
:1045960078D2677F011236B950077F011209418030
:1045A6005F7C007DA0D2677F011236B950117D076E
:1045B6007F061262A0500875450112781080417C72
:1045C600007DA8C2677F011236B950197D057F01AB
:1045D6001262A050107F061276235002D2087F0185
:1045E600124678801B7C007DB0C2677F011236B907
:1045F600500E7F061276235002D2087F011250BB5E
:10460600E4F54CAF4CEF3395E0FEEF7803C333CEC1
:1046160033CED8F92400F58274013EAD82FCD26710
:104626007F011236B95038754501AF4CEF3395E02E
:10463600FE74A02FF58274063EF583E0FFC007AF37
:104646004CEF3395E0FEEF7805C333CE33CED8F981
:1046560024F0F58274103EAD82FCD007126F8205FD
:104666004CC3E54C648094A84099C25BC265126D48
:014676008DB6
:014677002220
:104453007F061276235002C2087D017F061262A0F6
:10446300503D7C007D88C2677F021236B9500BD263
:10447300097F02121F58C20980257C007D70D26714
:104483007F021236B95002800D7C007D78D2677F9F
:10449300021236B95009D2097F02120941C20990AA
:1044A300001FE030E1427C007DA0D2677F0212361C
:1044B300B950147D077F061262A0500B1278FC7569
:1044C3004502127810801E7C007DA8C2677F02120D
:1044D30036B950147D057F021262A0500B1278FC8E
:1044E3007F021246781279ED7D027F061262A05098
:1044F3006AE4F54CAF4CEF3395E0FEEF7803C3333A
:10450300CE33CED8F92400F58274013EAD82FCD2BD
:10451300677F021236B95038754502AF4CEF3395B9
:10452300E0FE74A02FF58274063EF583E0FFC0071A
:10453300AF4CEF3395E0FEEF7805C333CE33CED8DF
:10454300F924F0F58274103EAD82FCD007126F821D
:10455300054CC3E54C648094A84099C25CC26612C2
:024563006DE108
:014565002233
:1049A9007D037F061262A0503D7C007D90C2677F27
:1049B900031236B9500BD20E7F03121F58C20E8054
:1049C900257C007D70D2677F031236B95002800DB5
:1049D9007C007D78D2677F031236B95009D20E7FE9
:1049E90003120941C20E90001FE030E2427C007DB3
:1049F900A0D2677F031236B950147D077F06126271
:104A0900A0500B1278FC754503127810801E7C00AB
:104A19007DA8C2677F031236B950147D057F031242
:104A290062A0500B1278FC7F031246781279ED7D53
:104A3900047F061262A0506AE4F54CAF4CEF33953F
:104A4900E0FEEF7803C333CE33CED8F92400F582E4
:104A590074013EAD82FCD2677F031236B9503875B6
:104A69004503AF4CEF3395E0FE74A02FF582740631
:104A79003EF583E0FFC007AF4CEF3395E0FEEF78DA
:104A890005C333CE33CED8F924F0F58274103EAD88
:104A990082FCD007126F82054CC3E54C648094A850
:094AA9004099C25DC228126E356D
:014AB20022E1
:104AB3007D057F061262A0503D7C007D98C2677F12
:104AC300041236B9500BD20C7F04121F58C20C804B
:104AD300257C007D70D2677F041236B95002800DA9
:104AE3007C007D78D2677F041236B95009D20C7FDF
:104AF30004120941C20C90001FE030E3427C007DA8
:104B0300A0D2677F041236B950147D077F06126264
:104B1300A0500B1278FC754504127810801E7C009F
:104B23007DA8C2677F041236B950147D057F041235
:104B330062A0500B1278FC7F041246781279ED7D47
:104B4300067F061262A0506AE4F54CAF4CEF339532
:104B5300E0FEEF7803C333CE33CED8F92400F582D9
:104B630074013EAD82FCD2677F041236B9503875AA
:104B73004504AF4CEF3395E0FE74A02FF582740625
:104B83003EF583E0FFC007AF4CEF3395E0FEEF78CF
:104B930005C333CE33CED8F924F0F58274103EAD7D
:104BA30082FCD007126F82054CC3E54C648094A845
:094BB3004099C260C22A126E8909
:014BBC0022D6
:10702200BF010AC214C210C21CC2188025BF020AC4
:10703200C215C211C21DC2198018BF030AC216C2EC
:1070420012C21EC21A800BBF0408C217C213C21F8B
:10705200C21B90001FE0FF30E002D224EF30E102B9
:0E706200D225EF30E202D226EF30E302D22731
:0170700022FD
:106636008F4B7868E6C39450507130496E20596B81
:106646007D077F011262A0502B205E287868E670D5
:106656000D90063BE0B54B06203F03D23F22202F8C
:106666000D203F0A7F01127022753D02D22F90063F
:1066760034E0F5327D087F061262A0501990063F7D
:10668600E0B54B06205E03D265220534E534AE3311
:10669600700E0533800A0534E534AE3370020533D7
:0C66A60014F5828E83E54BF07868062224
:1063AB008F4B7869E6C394505078304D75205972F5
:1063BB007D077F021262A050327F021278AF502B02
:1063CB00205E287869E6700D90063BE0B54B062001
:1063DB004103D2412220300D20410A7F021270224C
:1063EB00753D02D230900634E0F5327D087F0612FF
:1063FB0062A0501990063FE0B54B06205E03D266B3
:10640B00220536E536AE35700E0535800A0536E5C4
:10641B0036AE357002053514F5828E83E54BF07878
:03642B00690622DD
:10642E008F4B786AE6C3945050783051752059726C
:10643E007D077F031262A050327F031278AF502B7C
:10644E00205E28786AE6700D90063BE0B54B06207C
:10645E004303D2432220310D20430A7F03127022C0
:10646E00753D02D231900634E0F5327D087F06127A
:10647E0062A0501990063FE0B54B06205E03D2286D
:10648E00220538E538AE37700E0537800A0538E537
:10649E0038AE377002053714F5828E83E54BF078EF
:0364AE006A062259
:1064B1008F4B786BE6C394505078305475205972E5
:1064C1007D077F041262A050327F041278AF502BF7
:1064D100205E28786BE6700D90063BE0B54B0620F8
:1064E1004503D2452220320D20450A7F0412702235
:1064F100753D02D232900634E0F5327D087F0612F6
:1065010062A0501990063FE0B54B06205E03D22AE7
:1065110022053AE53AAE39700E0539800A053AE5A9
:106521003AAE397002053914F5828E83E54BF07865
:036531006B0622D4
:1078FC0090001FE0FF30E004D208D220EF30E1040A
:10790C00D209D221EF30E204D20ED222EF30E304BE
:05791C00D20CD2232271
:1079ED00C220C221C222C22390001FE0FF30E1025B
:0F79FD00C209EF30E202C20EEF30E302C20C22E9
:105DEC008F4C304603025E88304803025E88304C8C
:105DFC0003025E88304F03025E887D017F011262D0
:105E0C00A05079E54CB401197D017F051262A050B8
:105E1C000C90065AE0FF7C087D30127384786C0677
:105E2C0022E54CB402177D027F051262A050489007
:105E3C00065BE0FF7C087D50127384803AE54CB41D
:105E4C00041A7D027F051262A0500C90065DE0FFE3
:105E5C007C087D90127384786C760622E54C640382
:105E6C00701E7D027F051262A0500C90065CE0FF54
:105E7C007C087D70127384786C760122E4786CF661
:015E8C0022F3
:107ABA00EF1FAA0670011ED39400EA9400400BE45B
:0A7ACA00FDEDC394C850E90D80F7EC
:017AD400228F
:105A96008F5D306B5BE55DB40111D22090001FE095
:105AA600F420E003305E44D2088040E55DB4021184
:105AB600D22190001FE0F420E103305E2ED209804F
:105AC6002AE55DB40311D22290001FE0F420E20320
:105AD600305E18D20E8014E55DB4040FD223900018
:105AE6001FE0F420E303305E02D20CAF5D026C3798
:105AF600E55DB40110C22090001FE0F420E0033001
:105B06005E41C20822E55DB40210C22190001FE08A
:105B1600F420E103305E2CC20922E55DB40310C215
:105B26002290001FE0F420E203305E17C20E22E549
:105B36005DB4040FC22390001FE0F420E303305E3F
:045B460002C20C2269
:105B4A008F5330695BE553B40111D22490001FE0F2
:105B5A00F420E003305E44D2088040E553B40211D9
:105B6A00D22590001FE0F420E103305E2ED2098096
:105B7A002AE553B40311D22690001FE0F420E20371
:105B8A00305E18D20E8014E553B4040FD227900069
:105B9A001FE0F420E303305E02D20CAF53026C37ED
:105BAA00E553B40110C22490001FE0F420E0033052
:105BBA005E41C20822E553B40210C22590001FE0DC
:105BCA00F420E103305E2CC20922E553B40310C26B
:105BDA002690001FE0F420E203305E17C20E22E591
:105BEA0053B4040FC22790001FE0F420E303305E91
:045BFA0002C20C22B5
:08290E008F538C548D558B563C
:10291600C267E55524FFF582E55434FFF583E0F5FB
:1029260058855582855483E0FFF559A3E0FEF55A94
:10293600EF14B40800505C90294B75F003A4C583CE
:1029460025F0C5837302296302296A0229710229C7
:102956007802297F02298602298D0229947557015A
:10296600D267802F755702D2678028755704D267C1
:102976008021755708D267801A755710D267801361
:10298600755720D267800C755740D26780057557FA
:1029960080D267EE24FE7003022A5B24F8605C2472
:1029A600096003022A6DE553B401059000208045B5
:1029B600E553B40205900021803BE553B40305902E
:1029C60000228031E553B404059000238027E553A7
:1029D600B40505900024801DE553B4060590002536
:1029E6008013E553B407059000268009E553640873
:1029F6007077900027E04557F0806EE553B40105E7
:102A06009000208045E553B40205900021803BE507
:102A160053B403059000228031E553B404059000B9
:102A2600238027E553B40505900024801DE553B4A3
:102A360006059000258013E553B40705900026800F
:102A460009E55364087022900027E0FFE557F4FE7D
:102A5600EF5EF08014E553B4080D855582855483E6
:102A6600E0FF1260F4C267C267206703022B63E5CA
:102A760053B40109900020E0FD7F208060E553B447
:102A86000209900021E0FD7F218052E553B403093D
:102A9600900022E0FD7F228044E553B404099000B3
:102AA60023E0FD7F238036E553B40509900024E03A
:102AB600FD7F248028E553B40609900025E0FD7FBC
:102AC60025801AE553B40709900026E0FD7F26808D
:102AD6000CE553B4080C900027E0FD7F277E00121A
:102AE60073C4D2AFD26BAF56125A96AD58E4FF12EA
:102AF6007793AD59E4FF127793E55AB401047D3814
:102B06008007E55AB40A077D367F06127793E553A8
:102B1600B4080312770F7D077F061262A0500B20C0
:102B26002908C208C209C20EC20C7D017F011262C9
:102B3600A04002C2087D017F021262A04002C209C3
:102B46007D017F031262A04002C20E7D017F041246
:0D2B560062A04002C20CC26BAF56125A962C
:012B6300224F
:045E8D008F538D544E
:105E9100D26BAF54125A96AF54126C37E553B4011A
:105EA100059000208044E553B40205900021803A1A
:105EB100E553B403059000228030E553B404059006
:105EC10000238026E553B40505900024801CE5538A
:105ED100B406059000258012E553B407059000260D
:105EE1008008E553B40806900027E0F555E55560B4
:105EF10025755701E4F556E55530E007AD57E4FF48
:105F0100127793E555C313F55505570556E556C365
:105F1100940840E3800E7D187F021277937D537FB2
:0B5F210002127793C26BAF54125A9625
:015F2C002252
:021F58008F4DAB
:101F5A00E54D6401701E754E1B754F10900080E0B0
:101F6A00F550E54F2550F582E4354EF583E0F552FC
:101F7A0078688069E54D6402701E754E1B754F6066
:101F8A00900088E0F550E54F2550F582E4354EF58E
:101F9A0083E0F55278698045E54D6403701E754EFD
:101FAA001B754FB0900090E0F550E54F2550F58233
:101FBA00E4354EF583E0F552786A8021E54DB404A4
:101FCA001F754E1C754F00900098E0F550E54F259F
:101FDA0050F582E4354EF583E0F552786BE6F5511B
:101FEA00E55214B4090040030222F790200375F069
:101FFA0003A4C58325F0C5837302201E0220710243
:10200A0020C402211702216A0221BD0222100222E3
:10201A00610222B1E54F2550F582E4354EF583A3DE
:10202A00E0B40A18E5502402FFE433FEE551B5078F
:10203A000BE4B50607AD4D7F01022286AF507E0044
:10204A00EF2403FDEE33FCE5516D7001EC600302F1
:10205A0022F7EF254FFFEE354ECF2401FDE43FFC7A
:10206A00AB4D7F010222AEE54F2550F582E4354E95
:10207A00F583A3E0B40A18E5502402FFE433FEE531
:10208A0051B5070BE4B50607AD4D7F02022286AFB4
:10209A00507E00EF2403FDEE33FCE5516D7001EC38
:1020AA0060030222F7EF254FFFEE354ECF2401FDE4
:1020BA00E43FFCAB4D7F020222AEE54F2550F5828C
:1020CA00E4354EF583A3E0B40A18E5502402FFE490
:1020DA0033FEE551B5070BE4B50607AD4D7F0302A4
:1020EA002286AF507E00EF2403FDEE33FCE5516DEE
:1020FA007001EC60030222F7EF254FFFEE354ECF59
:10210A002401FDE43FFCAB4D7F030222AEE54F25DF
:10211A0050F582E4354EF583A3E0B40A18E550245D
:10212A0002FFE433FEE551B5070BE4B50607AD4DF2
:10213A007F04022286AF507E00EF2403FDEE33FCBB
:10214A00E5516D7001EC60030222F7EF254FFFEEB7
:10215A00354ECF2401FDE43FFCAB4D7F040222AE95
:10216A00E54F2550F582E4354EF583A3E0B40A180D
:10217A00E5502402FFE433FEE551B5070BE4B5064A
:10218A0007AD4D7F05022286AF507E00EF2403FD86
:10219A00EE33FCE5516D7001EC60030222F7EF2586
:1021AA004FFFEE354ECF2401FDE43FFCAB4D7F05DA
:1021BA000222AEE54F2550F582E4354EF583A3E0C1
:1021CA00B40A18E5502402FFE433FEE551B5070BC3
:1021DA00E4B50607AD4D7F06022286AF507E00EFBA
:1021EA002403FDEE33FCE5516D7001EC600302221D
:1021FA00F7EF254FFFEE354ECF2401FDE43FFCAB50
:10220A004D7F060222AEE54F2550F582E4354EF5A4
:10221A0083A3E0B40A17E5502402FFE433FEE55134
:10222A00B5070AE4B50606AD4D7F07804FAF507E6D
:10223A0000EF2403FDEE33FCE5516D7001EC600301
:10224A000222F7EF254FFFEE354ECF2401FDE43F82
:10225A00FCAB4D7F07804DE54F2550F582E4354EA6
:10226A00F583A3E0B40A18E5502402FFE433FEE53F
:10227A0051B5070BE4B50607AD4D7F08025E8DAF79
:10228A00507E00EF2403FDEE33FCE5516D7001EC46
:10229A00705BEF254FFFEE354ECF2401FDE43FFC86
:1022AA00AB4D7F0802290EE54F2550F582E4354EE5
:1022BA00F583A3A3E07036E54F2550F582E4354E49
:1022CA00F583A3E024F96008147022AF4D027888E0
:1022DA00D26B7F01125A96AF4D126C377D5E7F0228
:0D22EA00127793C26B7F01125A961259E1D0
:0122F70022C4
:0436B9008C4D8D4E59
:1036BD00054EE54E7002054D14F5828C83E0F970D0
:1036CD000302385BBF010875331B753410801FBFB3
:1036DD00020875351B7536608014BF030875371BDE
:1036ED007538B08009BF040675391C753A0020671E
:1036FD00030237C1BF01087868E6696002C322BFC3
:10370D0002087869E6696002C322BF0308786AE699
:10371D00696002C322BF0408786BE6696002C322A8
:10372D00E4FEEEC39940030237BFEF6401701CE560
:10373D004E2EF582E4354DF583E0FDE5342EF58210
:10374D00E43533F583E06D6002C322EF6402701C33
:10375D00E54E2EF582E4354DF583E0FDE5362EF58B
:10376D0082E43535F583E06D6002C322EF640370AA
:10377D001CE54E2EF582E4354DF583E0FDE5382E42
:10378D00F582E43537F583E06D6002C322EF640402
:10379D00701CE54E2EF582E4354DF583E0FDE53ADE
:1037AD002EF582E43539F583E06D6002C3220E02F9
:1037BD00372FD32230670302385CE4FEEEC3994005
:1037CD0003023859EF6401701CE54E2EF582E43585
:1037DD004DF583E0FDE5342EF582E43533F583E0D8
:1037ED006D6065C322EF6402701CE54E2EF582E418
:1037FD00354DF583E0FDE5362EF582E43535F5835F
:10380D00E06D6044C322EF6403701CE54E2EF5821B
:10381D00E4354DF583E0FDE5382EF582E43537F5D9
:10382D0083E06D6023C322EF6404701CE54E2EF51A
:10383D0082E4354DF583E0FDE53A2EF582E4353928
:0F384D00F583E06D6002C3220E0237C9D322C398
:01385C002249
:102B640090001FE0540FF55CB4010BE53EB4010383
:102B7400D21422C21422E55C6403702AE53EB40137
:102B840006D214D2108004C214C210E53EB402115D
:102B9400D2157D017F071262A04003022D7FD2115E
:102BA40022C215C21122E55C6405702AE53EB40117
:102BB40006D214D21C8004C214C21CE53EB4031114
:102BC400D2167D027F071262A04003022D7FD21E1F
:102BD40022C216C21E22E55C6409702AE53EB401D5
:102BE40006D214D2188004C214C218E53EB40411EB
:102BF400D2177D037F071262A04003022D7FD21BF0
:102C040022C217C21B22E55C6407704EE53EB40184
:102C140008D214D210D21C8006C214C210C21CE501
:102C24003EB40211D2157D017F071262A05002D278
:102C340011D21D8006C215C211C21DE53EB4031394
:102C4400D216D2127D027F071262A04003022D7FAA
:102C5400D21E22C216C212C21E22E55C640B704E42
:102C6400E53EB40108D214D210D2188006C214C2B0
:102C740010C218E53EB40211D2157D017F0712621D
:102C8400A05002D211D2198006C215C211C219E590
:102C94003EB40413D217D2137D037F071262A040FF
:102CA40003022D7FD21B22C217C213C21B22E55C72
:102CB400640D704BE53EB40108D214D21CD21880C6
:102CC40006C214C21CC218E53EB40311D2167D021A
:102CD4007F071262A05002D21ED21A8006C216C208
:102CE4001EC21AE53EB40413D217D21F7D037F0718
:102CF4001262A04003022D7FD21B22C2178078E506
:102D04005C640F7076E53EB4010AD214D210D21C72
:102D1400D2188008C214C210C21CC218E53EB40204
:102D240013D2157D017F071262A05002D211D21D69
:102D3400D2198008C215C211C21DC219E53EB403DE
:102D440013D216D2127D027F071262A05002D21E45
:102D5400D21A8008C216C212C21EC21AE53EB404B8
:102D640012D217D213D21F7D037F071262A0500B19
:0B2D7400D21B22C217C213C21FC21BD9
:012D7F002231
:100FB30090001FE0540FF55CB401167D017F011210
:100FC30062A0500A7F061276234003D20822C20889
:100FD30022E55C6403705BE53E640170257D017F5F
:100FE300011262A0500B7F061276234004D20880C0
:100FF30002C2087D017F021262A05003D20922C2FD
:101003000922E53E640260030214637D017F01123D
:1010130062A05004D2088002C2087D017F021262DE
:10102300A0500C7D017F071262A05003D20922C297
:101033000922E55C6405705BE53E640170257D0172
:101043007F011262A0500B7F061276234004D20860
:101053008002C2087D017F031262A05003D20E22D8
:10106300C20E22E53E640360030214637D017F0127
:101073001262A05004D2088002C2087D017F0312CD
:1010830062A0500C7D027F071262A05003D20E2291
:10109300C20E22E55C6409705BE53E640170257D48
:1010A300017F011262A0500B7F061276234004D207
:1010B300088002C2087D017F041262A05003D20C93
:1010C30022C20C22E53E640460030214637D017FA7
:1010D300011262A05004D2088002C2087D017F047D
:1010E3001262A0500C7D037F071262A05003D20C42
:1010F30022C20C22E55C640760030211B5E53E647D
:101103000170347D017F011262A0500B7F061276BD
:10111300234004D2088002C2087D017F021262A02C
:101123005004D2098002C2097D017F031262A050DC
:1011330003D20E22C20E22E53E640270367D017F89
:10114300011262A05004D2088002C2087D017F020E
:101153001262A0500D7D017F071262A05004D209D4
:101163008002C2097D017F031262A05003D20E22C6
:10117300C20E22E53E640360030214637D017F0116
:101183001262A05004D2088002C2087D017F0212BD
:1011930062A05004D2098002C2097D017F0312625A
:1011A300A0500C7D027F071262A05003D20E22C210
:1011B3000E22E55C640B6003021273E53E6401706A
:1011C300347D017F011262A0500B7F06127623400B
:1011D30004D2088002C2087D017F021262A050047B
:1011E300D2098002C2097D017F041262A05003D29A
:1011F3000C22C20C22E53E640270367D017F01128F
:1012030062A05004D2088002C2087D017F021262EC
:10121300A0500D7D017F071262A05004D209800205
:10122300C2097D017F041262A05003D20C22C20CBA
:1012330022E53E640460030214637D017F011262B0
:10124300A05004D2088002C2087D017F021262A06E
:101253005004D2098002C2097D017F041262A050AA
:101263000C7D037F071262A05003D20C22C20C2212
:10127300E55C640D6003021331E53E640170347D67
:10128300017F011262A0500B7F061276234004D225
:10129300088002C2087D017F031262A05004D20EAF
:1012A3008002C20E7D017F041262A05003D20C2281
:1012B300C20C22E53E640370367D017F011262A0F9
:1012C3005004D2088002C2087D017F031262A0503D
:1012D3000D7D027F071262A05004D20E8002C20E5F
:1012E3007D017F041262A05003D20C22C20C22E5BE
:1012F3003E640460030214637D017F011262A05007
:1013030004D2088002C2087D017F031262A0500448
:10131300D20E8002C20E7D017F041262A0500C7DAA
:10132300037F071262A05003D20C22C20C22E55C99
:10133300640F6003021463E53E640170437D017F23
:10134300011262A0500B7F061276234004D208805C
:1013530002C2087D017F021262A05004D2098002FA
:10136300C2097D017F031262A05004D20E8002C223
:101373000E7D017F041262A05003D20C22C20C2204
:10138300E53E640270457D017F011262A05004D2E4
:10139300088002C2087D017F021262A0500D7D0108
:1013A3007F071262A05004D2098002C2097D017F27
:1013B300031262A05004D20E8002C20E7D017F048C
:1013C3001262A05003D20C22C20C22E53E640370C9
:1013D300457D017F011262A05004D2088002C20839
:1013E3007D017F021262A05004D2098002C2097DEE
:1013F300017F031262A0500D7D027F071262A0508D
:1014030004D20E8002C20E7D017F041262A050033B
:10141300D20C22C20C22E53E640470447D017F019C
:101423001262A05004D2088002C2087D017F02121A
:1014330062A05004D2098002C2097D017F031262B7
:10144300A05004D20E8002C20E7D017F041262A05E
:10145300500C7D037F071262A05003D20C22C20CF2
:011463002266
:10798C007F011278AF5010C209C20EC20C7F0612D2
:10799C007623500CC208227F011278AF4002C20835
:0179AC0022B8
:107B09007F021278AF5007C209C20EC20C227F024F
:087B19001278AF4002C20922FC
:107B21007F031278AF5007C209C20EC20C227F0335
:087B31001278AF4002C20E22DF
:107B39007F041278AF5007C209C20EC20C227F041B
:087B49001278AF4002C20C22C9
:106A13000500050105030507050F051F051E051CD8
:106A2300051805100201040E040A03060101040BF4
:106A33000304040F020304010302040D0200020213
:106A43000300040904040305030701000303040707
:106A5300030104060402040C0516051500000615BF
:0E6A6300062A060C06380633061E0612061713
:10539200203737900640E004F519D3648094815099
:1053A2000302546CD3E5196480948F400375190F7E
:1053B20090063DE0FF123E6090063EE0F518E4F5EF
:1053C2001ED237C264C257C24A22304A60306416C3
:1053D200152EE52ED39400400302546CC2CAC26457
:1053E200D25785182E2230570E152EE52ED3940053
:1053F2005078C264C25722AF1C151CEF700BC24A10
:10540200E51825E0F52ED25722E51D30E005851876
:105412002E8008E51875F003A4F52EAF1D7801EF74
:1054220008800103D8FDF51DD264D2CA22D519081D
:10543200C237E4F53DC25822051E7440251EF5828E
:10544200E43406F583E025E02413F582E4346AF5BA
:1054520083E493540FF51C740193F51D700AD2571F
:0A546200E51825E025E0F52ED24AFA
:01546C00221D
:105FC60020371A90063DE0FF123E6090063EE0F54F
:105FD6001AE4F51ED237C264C257C24A22304A5961
:105FE600306413152EE52ED39400506BC2CAC264DA
:105FF600D257851A2E2230570E152EE52ED3940031
:106006005055C264C25722AF1C151CEF7007C24A16
:10601600C237F53D22E51D30E005851A2E8008E5DC
:106026001A75F003A4F52EAF1D7801EF0880010361
:10603600D8FDF51DD264D2CA22E53F25E02413F52A
:1060460082E4346AF583E493FA740193FBEA540F0D
:07605600F51CEBF51DD24A19
:01605D002220
:107BCE00C3EF648094A15008EF25E025E0F52E2246
:047BDE00E4F52E227A
:10755400BF010790063E7418F022BF020790063E52
:107564007412F022BF030590063E8014BF040790F6
:10757400063E740BF02290063EBF05047409F02207
:04758400740CF02271
:103E6000EF14B420004003023FB3903E7875F00396
:103E7000A4C58325F0C58373023ED8023EDF023E0F
:103E8000E6023EED023EF4023EFB023F02023F0923
:103E9000023F10023F17023F1E023F25023F2C0245
:103EA0003F33023F3A023F41023F48023F4F023F49
:103EB00056023F5D023F64023F6B023F72023F7950
:103EC000023F80023F87023F8E023F95023F9702EA
:103ED0003F9E023FA5023FAC75CB8E75CAC62275C8
:103EE000CB9575CA772275CB9B75CA692275CBA015
:103EF00075CABA2275CBA675CA332275CBAB75CA03
:103F0000632275CBB075CA022275CBB475CAA322E1
:103F100075CBB875CAFA2275CBBC75CAD82275CBD9
:103F2000C075CAA82275CBC475CA362275CBC775B1
:103F3000CA862275CBCA75CABC2275CBCD75CAB4E8
:103F40002275CBD075CA762275CBD375CA3022754F
:103F5000CBD575CAB22275CBD875CA132275CBDA08
:103F600075CA522275CBDC75CA7D2275CBDD75CA48
:103F70006E2275CBE075CA542275CBE275CA1B223E
:103F800075CBE375CAC32275CBE575CA5E2275CBC6
:103F9000E675CADA22801C75CBE875CA902275CB0B
:103FA000EA75CAD92275CBEC75CA092275CBED75B5
:0A3FB000CA292275CBE875CA412228
:10727600EFC39400403FEF9408503AE4FEEF75F0F8
:1072860008A42430F582E43400F583E5822EF582E5
:10729600E43583F583E0FCED75F008A424E8F58277
:1072A600E4341AF583E5822EF582E43583F583EC22
:0572B600F00EBE08C847
:0172BB0022B0
:1060F4008F5BE55B6405701D200A0DD20A7FF47E78
:1061040001127ABAC20A8074C20A7FF47E01127A3A
:10611400BAD20A8067E55B6406701D200B0DD20BB2
:106124007FF47E01127ABAC20B800BC20B7FF47E1D
:1061340001127ABAD20B8044E55B6407701D200F0C
:106144000DD20F7FF47E01127ABAC20F800BC20FF8
:106154007FF47E01127ABAD20F8021E55B64087065
:1061640022200D0DD20D7FF47E01127ABAC20D8069
:106174000BC20D7FF47E01127ABAD20D7FF47E0138
:04618400127ABA22AF
:104FC200A233B330B401B350357D017F081262A021
:104FD2005027A233B35010A2B4B3500B900652E044
:104FE200FF7C077D30800F30330F30B40C900653B6
:104FF200E0FF7C077D50127384A2B4B39233A234D3
:10500200B330B501B350357D027F081262A050273C
:10501200A234B35010A2B5B3500B900654E0FF7CFB
:10502200077D70800F30340F30B50C900655E0FFCD
:105032007C077D90127384A2B5B39234A235B3304B
:10504200B701B350357D037F081262A05027A23505
:10505200B35010A2B7B3500B900656E0FF7C077D09
:10506200B0800F30350F30B70C900657E0FF7C0749
:105072007DD0127384A2B7B39235A236B330B60193
:10508200B350357D047F081262A05027A236B35078
:1050920010A2B6B3500B900658E0FF7C077DF0805B
:1050A2000F30360F30B60C900659E0FF7C087D10A9
:0950B200127384A2B6B3923622F7
:10770F00900027E0FF30E404D20A8002C20AEF3073
:10771F00E504D20B8002C20BEF30E604D20F8002D9
:0B772F00C20FEF30E703D20D22C20DA5
:01773A00222C
:1074B40090063CE0FF602E20370F6029123E60D218
:1074C400CAD237D264752E1422E52ED39400400319
:1074D400152E22206408D2CA752E14D26422C2CA80
:0674E400752E7DC264223A
:1074EA002037127F1C123E60D2CAD237D264752E60
:1074FA0064751B3C22E52ED394004003152E22AF5F
:10750A001B151BD3EF648094804004752E6422C23D
:04751A0037E4F53D20
:01751E00224A
:104DC60020371C754006E53E75F008A424E8F582F8
:104DD600E4341AF583E06003D23722E4F53D22E598
:104DE6002ED394004003152E22C2CA1540E5401466
:104DF6007003024E8614607414604114602F1460B0
:104E060003024EBEE53E75F008A424E8F582E434BC
:104E16001AF583E0FF7003F53D22123E60E53E750C
:104E2600F008A424E9F582E4341A024EB4E53E758E
:104E3600F008A424EAF582E4341A803D7408441B81
:104E46007003F53D22E53E75F008A424EBF582E4F7
:104E5600341AF583E0FF7002805F123E60E53E750E
:104E6600F008A424ECF582E4341A8042E53E75F09D
:104E760008A424EDF582E4341AF583E0FF027BCE24
:104E86007420441B7003F53D22E53E75F008A4240A
:104E9600EEF582E4341AF583E0FF7002801B123EC1
:104EA60060E53E75F008A424EFF582E4341AF58334
:104EB600E0FF127BCED2CA22E4F53DC2CAC2372237
:10758800E53D14601C14601C14601C14601F14601A
:107598001F2405701EC2CAC237C264C257E4F54030
:1075A80022024DC60274B4125392D258220274EACF
:0475B800125FC62276
:1076B500E52365437004E5226542601F8522428506
:1076C5002343C2A4D2A5C2A6C2A700AF23127B67DB
:0D76D500E522FF127B6700D2A7D322C3225B
:107A8200E52465446014852444D2A4D2A5C2A6C2CA
:0C7A9200A7AF24127B67D2A7D322C32227
:107A9E00E521653C601485213CD2A4C2A5C2A6C2D4
:0C7AAE00A7AF21127B67D2A7D322C3220E
:10422100E4F54CF54D754E1E754FFF854D82854C5D
:1042310083E0F5506350FFE550F0E06550600312F4
:104241007C5E6350FF854D82854C83E550F0E065CF
:10425100506003127C5E054DE54D7002054CE54F43
:10426100154F7002154ED3E54F9400E54E94005062
:10427100BAE4F54CF54DF54EF54FE54D254FF58278
:10428100E54C354EF583E4F0054FE54F7002054EE0
:10429100B4FFE7E54EB41EE275985A758921758819
:1042A10045758845758DE775878075C90275331B1E
:1042B10075341075351B75366075371B7538B075DB
:1042C100391C753A0075B701D2A9D2A8D2AA9006B5
:1042D10000E0FFA3E0901CE0CFF0A3EFF090060216
:1042E100E0FFA3E0901CE2CFF0A3EFF0900604E022
:1042F100FFA3E0901CE4CFF0A3EFF0900606E0FFEF
:10430100A3E0901CE6CFF0A3EFF0901CFA7417F035
:10431100A37499F0901CFC7417F0A37499F0901C8D
:10432100FE7417F0A37499F0901D007417F0A37434
:0943310099F0D291D2AF1277BDD0
:01433A002260
:027C5E0080FEA6
:10762300C2AFC284D285BF060AC286E580A2E192B8
:107633006B8018BF070AC286E580A2E2926B800BBB
:10764300BF0808C286E580A2E3926BD286D2AFA2BE
:017653006BCB
:017654002213
:1062A000BF0107900020E0FE8048BF020790002158
:1062B000E0FE803EBF0307900022E0FE8034BF0472
:1062C00007900023E0FE802ABF0507900024E0FE2F
:1062D0008020BF0607900025E0FE8016BF070790CC
:1062E0000026E0FE800CBF0807900027E0FE800239
:1062F000E4FEBD0103EE1322BD0204EEA2E122BDC5
:106300000304EEA2E222BD0404EEA2E322BD0504D2
:10631000EEA2E422BD0604EEA2E522BD0704EEA231
:07632000E622BD0802EE3386
:016327002253
:0250BB008F4D17
:1050BD009000B0E0F54EE54D64017037E54E2402E9
:1050CD00FFE433FE7868E66F7001EE60030251B0C5
:1050DD007410254EF582E4341BAF82F5508F51D2FA
:1050ED006B7F01125A96127A4812385DC26B7F019E
:1050FD000251ADE54D64027037E54E2402FFE433F5
:10510D00FE7869E66F7001EE60030251B0746025A0
:10511D004EF582E4341BAF82F5508F51D26B7F0276
:10512D00125A96127A4812385DC26B7F020251AD47
:10513D00E54D64037033E54E2402FFE433FE786AD7
:10514D00E66F7001EE705C74B0254EF582E4341B91
:10515D00AF82F5508F51D26B7F03125A96127A4857
:10516D0012385DC26B7F038037E54D64047034E502
:10517D004E2402FFE433FE786BE66F7001EE702370
:10518D007400254EF582E4341CAF82F5508F51D258
:10519D006B7F04125A96127A4812385DC26B7F04E7
:0351AD00125A96FD
:0151B00022DC
:04385D008F4FE4FDA8
:023861008D5781
:1038630075F020EFA42460F582E5F03403AF82F510
:103873005A8F5BF583E0F558D3940050030239E97E
:10388300E558941040030239E9E557704C7FF47E04
:1038930001127ABAE55825E0F558755901E558241F
:1038A30001FFE433FEC3E5599FEE6480F87480980A
:1038B30040030239E9E55B2559F582E4355AF5837E
:1038C300E0FFE55B2559F582E4355AF583A3E0FD76
:1038D3001277930559055980C4E5576401707AC27C
:1038E3002B7FF47E01127ABAE55825E0F558755915
:1038F30001E5582401FFE433FEC3E5599FEE6480DC
:10390300F874809840030239E9E55B2559F582E4B0
:10391300355AF583E0FFE55B2559F582E4355AF521
:1039230083A3E0FD12779390001FE0FF30E00630A1
:103933004903C22022EF30E106304D03C22122EFBA
:1039430030E206305103C22222EF30E30630540343
:10395300C22322055905598098E557640260030282
:1039630039E9C22BC22CC22DC22E7FF47E01127AFA
:10397300BAE55825E0F558755901E5582401FFE4E7
:1039830033FEC3E5599FEE6480F87480985057E581
:103993005B2559F582E4355AF583E0FFE55B25594C
:1039A300F582E4355AF583A3E0FD12779390001F67
:1039B300E030E005303902802290001FE030E1055D
:1039C300303A02801690001FE030E205303B02805F
:1039D3000A90001FE030E308303C05C22002730167
:0639E3000559055980940E
:0139E90022BB
:024678008F4D64
:10467A00C2679000A8E0FFE54DB401167868E6FE2F
:10468A00D39F400EEE9FF55074102FF582E4341B31
:10469A00804FE54DB402167869E6FED39F400EEED0
:1046AA009FF55074602FF582E4341B8034E54DB4D5
:1046BA000316786AE6FED39F400EEE9FF55074B05B
:1046CA002FF582E4341B8019E54DB4041C786BE69F
:1046DA00FED39F4014EE9FF55074002FF582E43408
:1046EA001CAF82F5518F52D267206703024788D2E6
:1046FA006BAF4D125A967FF47E01127ABA7D207FF3
:10470A00051277937D1A7F081277937FC87E00126D
:10471A007ABAE4F54EE54EC39550505B0552E55220
:10472A00AE517002055114F5828E83E0F54F603662
:10473A0024F5601414601714601A14601D146020A4
:10474A0024057028E4FD80277D5F7F0780227D5E37
:10475A007F06801C7D0A7F0280167D327F028010D0
:10476A007D467F02800A7D0A7F038004AD4FE4FF05
:0E477A00127793054E809EC26BAF4D125A9679
:01478800220E
:1078100030290F900671E0FF7C0B7D10127384B24B
:107820002922202912900670E0FF7C0A7DF0127355
:0878300084B229E4786CF62211
:10605E007D3F7F091277937D507F081277939000D2
:10606E000EE493FDE4FF1277937D5B7F0612779328
:10607E0090000FE493FDE4FF127793900010E493E9
:10608E00FDE4FF127793900011E49324BFB408004F
:10609E0050539060AE75F003A4C58325F0C583738D
:1060AE000260C60260CA0260CE0260D40260DA02EA
:1060BE0060E00260E60260EC7D0A80067D328002BE
:1060CE007D467F02801C7D0A7F0380167D287F031C
:1060DE0080107D467F03800A7D0A7F0480047D2820
:0660EE007F0412779322EB
:107888008F53D26B125A967D4B7F021277937D04E9
:10789800E4FF1277937D387F0412779312605EC2FB
:0778A8006BAF53125A962248
:0B7A4800855182855083E0FFA3E0FD24
:107A5300BF0A02E4FFBD0A02E4FDEF75F00AA42D9C
:027A6300FF2200
:10546D00C267D208D2207FF47E01127ABA7D2E7FD8
:10547D00031277937D607F02127793C208C22012C8
:10548D0033467F0812762340030255393049F01216
:10549D0033462049FA7868E6640770427E007F70D3
:1054AD0075331B7534108F828E837407F07D01E583
:1054BD00342DF582E43533F583E58224FFF582E55D
:1054CD008334FFF583E0F9EF2DF582E43EF583E9B2
:1054DD00F00DBD08DAD2677F647E00127ABA7F08BC
:1054ED00127623504720670302546FD208D2207FD3
:1054FD00F47E01127ABA7D607F021277937D327F3E
:10550D00061277937D1E7F05127793C208C2207C09
:10551D00007D707B087F787E001268167F081276FA
:10552D002350097F327E00127ABA80F0126D8D7F82
:06553D00647E00127ABA40
:015543002245
:1077E700E4F53DC258C258F532302F05C22FC23FCB
:1077F70022303005C230C24122303105C231C24386
:0978070022303204C232C24522D3
:10433B007580FFC286E580540FFFC285E580C454AB
:10434B00F04FF520D2867D027F011262A040107DD6
:10435B00037F011262A04007300004D23980287D10
:10436B00027F011262A0500A300007300104D239DB
:10437B0080157D037F011262A0500A2000033001DB
:10438B0004D2398002C2397D027F021262A0401032
:10439B007D037F021262A04007300204D23A8028CC
:1043AB007D027F021262A0500A300207300304D252
:1043BB003A80157D037F021262A0500A200203305F
:1043CB000304D23A8002C23A7D027F031262A040FC
:1043DB00107D037F031262A04007300404D23B80A0
:1043EB00287D027F031262A0500A300407300504B7
:1043FB00D23B80157D037F031262A0500A20040379
:10440B00300504D23B8002C23B7D027F041262A0C6
:10441B00400F7D037F041262A04006300603D23C9E
:10442B00227D027F041262A050093006063007037A
:10443B00D23C227D037F041262A050092006033078
:07444B000703D23C22C23C32
:014452002247
:10334600202B6EC25A20391C205019901CFAE070AE
:1033560002A3E0700B7D067F011262A05002D247E5
:10336600C249804D30392130501E901CE0E0700279
:10337600A3E0700B7D087F011262A05002D23D309F
:103386006502D25BD2498029303908205005126D7A
:103396008D801E20391B305018D25AC249C250C2E5
:1033A60014C210C21CC21812798C7868E66002D268
:1033B6005B202C71203A1C205319901CFCE07002F3
:1033C600A3E0700B7D067F021262A05002D24BC2B0
:1033D6004D8052303A28305325901CE2E07002A30B
:1033E600E070127D087F021262A050097F021278F7
:1033F600AF5002D23E306602D25BD24D8027303AC1
:1034060008205305126DE1801C203A19305316C26C
:103416004DC253C215C211C21DC219127B09786969
:10342600E66002D25C202D71203B1C205519901CB1
:10343600FEE07002A3E0700B7D067F031262A050CF
:1034460002D24EC2518052303B28305525901CE4A2
:10345600E07002A3E070127D087F031262A050099B
:103466007F031278AF5002D240302802D25BD2518D
:103476008027303B08205505126E35801C203B19ED
:10348600305516C251C255C216C212C21EC21A12F7
:103496007B21786AE66002D25D202E6D203C1B20DF
:1034A6005618901D00E07002A3E0700B7D067F04A5
:1034B6001262A05002D252C25422303C2730562407
:1034C600901CE6E07002A3E070127D087F04126291
:1034D600A050097F041278AF5002D242302A02D29D
:1034E6005BD25422303C06205603026E89203C19DA
:1034F600305616C254C256C217C213C21FC21B127E
:0A3506007B39786BE66002D2602288
:047C57001251B122F3
:1051B10090001FE0540FFFBF010B304906203D0353
:1051C100025278C322EF64037014304906203D0374
:1051D100025278304D06203E03025283C322EF640F
:1051E100057014304906203D0302527830510620E3
:1051F100400302528EC322EF640970133049052027
:105201003D028073305406204203025299C322EFBB
:105211006407701A304905203D02805B304D05203E
:105221003E02805E3051052040028061C322EF645E
:105231000B701A304905203D02803C304D05203E5F
:1052410002803F305405204202804DC322EF640D9D
:10525100701A304905203D02801D30510520400261
:10526100802B305405204202802EC322EF640F7040
:105271002E304908203D05753E01D322304D0820CE
:105281003E05753E02D322305108204005753E038C
:10529100D322305408204205753E04D322C322C3D1
:0152A10022EA
:1078AF00BF010690001FE01322BF020790001FE0E8
:1078BF00A2E122BF030790001FE0A2E222BF04064D
:0778CF0090001FE0A2E3227C
:106D8D007868E6602275331B753410E4FFE5342F07
:106D9D00F582E43533F583E4F00FBF50F075331B06
:106DAD00753410E47868F6900600E0FFA3E0901CBF
:106DBD00E0CFF0A3EFF0900608E0FFA3E0901CFAFF
:106DCD00CFF0A3EFF0C246C247C25FC23DC265C25B
:036DDD003FD25052
:016DE0002290
:106DE1007869E6602275351B753660E4FFE5362F5C
:106DF100F582E43535F583E4F00FBF50F075351BAE
:106E0100753660E47869F6900602E0FFA3E0901C15
:106E1100E2CFF0A3EFF090060AE0FFA3E0901CFCA4
:106E2100CFF0A3EFF0C248C24BC261C23EC266C2FC
:036E310041D253F8
:016E3400223B
:106E3500786AE6602275371B7538B0E4FFE5382FB0
:106E4500F582E43537F583E4F00FBF50F075371B55
:106E55007538B0E4786AF6900604E0FFA3E0901C6C
:106E6500E4CFF0A3EFF090060CE0FFA3E0901CFE4A
:106E7500CFF0A3EFF0C24CC24EC262C240C228C2DC
:036E850043D255A0
:016E880022E7
:106E8900786BE6602275391C753A00E4FFE53A2F04
:106E9900F582E43539F583E4F00FBF50F075391CFC
:106EA900753A00E4786BF6900606E0FFA3E0901CC3
:106EB900E6CFF0A3EFF090060EE0FFA3E0901D00EF
:106EC900CFF0A3EFF0C24FC252C263C242C22AC27C
:036ED90045D25649
:016EDC002293
:1059E100C208C209C20EC20C127A9EC267D25EE41C
:1059F100F53D7FE87E03127ABAC298C2AF75567F31
:105A0100755596755498755300785374FF1259C3A0
:105A1100E4FBFAF9F8C31259B0504430983E120031
:105A210006127C19EF14601824F0602624C1600B63
:105A310024F670287F06127C4780211271E6801CB3
:105A41007F06127C471275BC12770F1270BED267A7
:105A5100800A7F06127C471267A5D2673067AAE4E5
:105A6100786CF6D26B7F01125A967F01126C377DEA
:105A7100467F021277937D1E7F071277937D147FF5
:105A8100081277937D327F03127793C26B7F0112E5
:045A91005A96C25E01
:015A950022EE
:1067A500756701756500756620E4F5577F02127CF3
:1067B50047E5672402F559AF67127C47E4F558E5CC
:1067C500662558F582E43565F583E0FF127C47E5DB
:1067D500662558F582E43565F583E02559F55905B3
:1067E50058E558C3948040D7AF59127C477F0312B0
:1067F5007C47127C4FEF641560160567748025662B
:10680500F566E43565F5650557E557C39435409C50
:016815002260
:1075BC00756701756500756620E4F5571276E25023
:1075CC00077F06127C4780057F15027C4705677490
:1075DC00802566F566E43565F5650557E557C39472
:0375EC003540D94E
:0175EF002279
:1076E200E4F558127C4F74502558F582E4341CF5A9
:1076F20083EFF00558E558C3948440E7127B7D90F0
:0C7702001CD2E0B507051279ADD322C3FC
:01770E002258
:1079AD00E4FF74522FF582E4341CF583E0FEE566A6
:0F79BD002FF582E43565F583EEF0000FBF80E310
:0179CC002298
:107B7D00E4FFFE74502EF582E4341CF583E02FFFF4
:047B8D000EBE82EFB7
:017B910022D1
:1071E600E4F557F55D755CE0755B93755A04F559E2
:1071F600785974FF1259C3E4FBFAF9F8C31259B06F
:1072060050253098EB1200068F58E5586404601735
:10721600AF5D055D74502FF582E4341CF583E558A7
:07722600F02557F55780C960
:01722D00223E
:04000600AF99C29854
:01000A0022D3
:087C47003099FDC2998F9922CA
:077C4F003098FDAF99C298C7
:017C5600220B
:105BFE000701020304050607070706050403020151
:105C0E0003010A0A03020A0A03030A0A03040A0A20
:105C1E00030307050303020503070A0A04024B00E8
:105C2E00040438072E03024B0004043802055F00FB
:105C3E000302055F000402055F000502055F000612
:105C4E0002055F000702055F000802055F000902FA
:105C5E00055F000A02055F000B02055F000C0205DE
:105C6E005F000D02055F000E02055F000F02055F6B
:105C7E00001002055F001102055F001204072E08D6
:105C8E00260640033204072E082606400253080C4F
:075C9E000A1D040000241B95
:10001600C2AF9000207491F09000217481F090009E
:1000260022F0900023F09000247403F090002574D1
:10003600BFF09000267418F0900027740FF090001F
:10004600307409F0A37403F0E4A3F0A37410F0A3D2
:100056007403F0E4A3F0A37415F0A37403F0A3747F
:1000660015F0A37403F0E4A3F0A37410F0A37403D3
:10007600F0E4A3F0A37409F0A37403F0A37415F0DD
:10008600A37403F0A314F0A3741AF0A37403F0E4AA
:10009600A3F0A3F0A3F0A3741AF0A37403F0A314BF
:1000A600F0A37415F0A37403F0E4A3F0A3F0A3F097
:1000B6007E5C7F0E7C007D807B041273437E5C7FBA
:1000C600127C007D887B041273437E5C7F167C0065
:1000D6007D907B041273437E5C7F1A7C007D987B47
:1000E600041273437E5C7F227C007DA07B04127326
:1000F600437E5C7F1E7C007DA87B041273437E5C7E
:100106007F267C007DB07B041273437E5B7FFE7C82
:10011600007D707B081273437E5C7F067C007D78D1
:100126007B081273437E5C7F2A7C037D807B0912E9
:1001360073437E5C7F337C037DA07B071273437E13
:100146005C7F3A7C037DC07B051273437E5C7F3FF8
:100156007C037DE07B051273437E5C7F447C047DDB
:10016600007B051273437E5C7F497C047D207B0502
:100176001273437E5C7F4E7C047D407B0512734385
:100186007E5C7F537C047D607B051273437E5C7FBF
:10019600587C047D807B051273437E5C7F5D7C0406
:1001A6007DA07B051273437E5C7F627C047DC07BF1
:1001B600051273437E5C7F677C047DE07B051273CA
:1001C600437E5C7F6C7C057D007B051273437E5C01
:1001D6007F717C057D207B051273437E5C7F767C78
:1001E600057D407B051273437E5C7F7B7C057D60CD
:1001F6007B051273437E5C7F807C057D807B0512C8
:1002060073437E5C7F857C057DA07B051273437EF0
:100216005C7F8A7C057DC07B091273437E5C7F937D
:100226007C057DE07B09127343900600E4F0A3741D
:10023600B4F0900602E4F0A374B4F0900604E4F07F
:10024600A374B4F0900606E4F0A374B4F090061814
:100256007401F0A374E0F090061AE4F0A37478F049
:1002660090061EE4F0A3743CF09006087402F0A316
:100276007458F090060A7402F0A37458F090060CB5
:100286007402F0A37458F090060E7402F0A374582A
:10029600F09006107401F0A3742CF090061274020C
:1002A600F0A37458F09006147403F0A37484F090CD
:1002B60006167404F0A374B0F07407900620F0A339
:1002C600F0900622F0A3F090061C7402F0A3745876
:1002D600F0900630740AF09006317428F0900633D8
:1002E600740AF0900634F09006327405F07E5C7F56
:1002F6009C7C067D407B0912734390063D7417F083
:1003060090063E740CF090063C7419F0E490063F9B
:10031600F090063B740CF09006527401F090073092
:100326007469F0A37411F09006537401F0900750AD
:100336007469F0A37410F09006547401F09007707D
:100346007469F0A37421F09006557401F09007903B
:100356007469F0A37420F09006567401F09007B00B
:100366007469F0A37431F09006577401F09007D0C9
:100376007469F0A37430F09006587401F09007F099
:100386007469F0A37441F09006597401F090081056
:100396007469F0A37440F090065A7401F090083026
:1003A6007462F0A37411F0A37432F0A37401F0A385
:1003B6007450F0A37410F090065B7401F09008502E
:1003C6007461F0A37420F0A37462F0A37411F0A317
:1003D6007432F0A37402F0A37450F0A37410F0907A
:1003E600065C7401F09008707451F0A37411F0A3C8
:1003F6007433F0A3E4F0A37451F0A37410F09006E4
:100406005D7401F09008907462F0A37411F0A37407
:1004160030F0A37402F0A37462F0A37410F0900697
:100426005E7401F09008B07451F0A37411F0A374D7
:1004360041F0A37410F0A37451F0A37410F0900669
:100446005F7401F09008D07451F0A37411F0A37496
:1004560034F0A37414F0A37451F0A37410F0900652
:10046600607401F09008F07451F0A37411F0A37455
:1004760034F0A37418F0A37451F0A37410F090062E
:10048600617401F09009107451F0A37411F0A37413
:1004960034F0A37428F0A37451F0A37410F09006FE
:1004A600627401F09009307462F0A37411F0A374C1
:1004B60030F0A37403F0A37462F0A37410F09006F6
:1004C600637401F09009507462F0A37411F0A37480
:1004D60030F0A37404F0A37462F0A37410F09006D5
:1004E600647401F09009707462F0A37411F0A3743F
:1004F60060F0A37401F0A37495F0A3743DF0A374A7
:1005060090F0A37401F0A37498F0A37426F0A3747A
:1005160096F0A37440F0A37462F0A37410F0A37471
:1005260061F0A37470F09006657401F09009907400
:1005360062F0A37411F0A37460F0A37401F0A374C5
:1005460095F0A3743DF0A37490F0A37401F0A37426
:1005560096F0A37438F0A37462F0A37410F09006BA
:10056600667401F09009B07462F0A37411F0A3747C
:1005760060F0A37401F0A37495F0A3743DF0A37426
:1005860090F0A37402F0A37498F0A37426F0A374F9
:1005960096F0A37440F0A37462F0A37410F0A374F1
:1005A60061F0A37470F09006677401F09009D0743E
:1005B60062F0A37411F0A37460F0A37401F0A37445
:1005C60095F0A3743DF0A37490F0A37402F0A374A5
:1005D60096F0A37438F0A37462F0A37410F090063A
:1005E600687401F09009F07462F0A37411F0A374BA
:1005F60060F0A37401F0A37495F0A3743DF0A374A6
:1006060090F0A37403F0A37498F0A37426F0A37477
:1006160096F0A37440F0A37462F0A37410F0A37470
:1006260061F0A37470F09006697401F0900A10747A
:1006360062F0A37411F0A37460F0A37401F0A374C4
:1006460095F0A3743DF0A37490F0A37403F0A37423
:1006560096F0A37438F0A37462F0A37410F09006B9
:100666006A7401F0900A307462F0A37411F0A374F6
:1006760060F0A37401F0A37495F0A3743DF0A37425
:1006860090F0A37404F0A37498F0A37426F0A374F6
:1006960096F0A37440F0A37462F0A37410F0A374F0
:1006A60061F0A37470F090066B7401F0900A5074B8
:1006B60062F0A37411F0A37460F0A37401F0A37444
:1006C60095F0A3743DF0A37490F0A37404F0A374A2
:1006D60096F0A37438F0A37462F0A37410F0900639
:1006E6006C7401F0900A707462F0A37411F0A37434
:1006F60060F0A37401F0A37430F0A37405F0A37442
:1007060062F0A37410F090066D7401F0900A907474
:1007160062F0A37421F0A37460F0A37401F0A374D3
:1007260030F0A37406F0A37462F0A37420F0900670
:100736006E7401F0900AB07462F0A37431F0A37481
:1007460060F0A37401F0A37430F0A37407F0A374EF
:1007560062F0A37430F090066F7401F0900AD074C2
:1007660062F0A37441F0A37460F0A37401F0A37463
:1007760030F0A37408F0A37462F0A37440F09006FE
:10078600707401F0900AF07464F0A37411F0A3740D
:1007960096F0A37432F0A37495F0A3741EF0A374BC
:1007A60098F0A3744BF0A37464F0A37410F0900651
:1007B600717401F0900B107464F0A37411F0A374BB
:1007C60096F0A37432F0A37495F0A3741EF0A3748C
:1007D60093F0A37418F0A37464F0A37410F0900659
:1007E600737401F0900B507462F0A37411F0A3744B
:1007F60060F0A37401F0A37495F0A3743DF0A374A4
:1008060090F0A37402F0A37497F0A37426F0A37477
:1008160093F0A37418F0A37462F0A37410F0A37499
:1008260070F0A37410F09006747401F0900B70745D
:1008360062F0A37411F0A37460F0A37401F0A374C2
:1008460095F0A3743DF0A37490F0A37403F0A37421
:1008560097F0A37426F0A37493F0A37418F0A3740E
:1008660062F0A37410F0A37470F0A37420F09006E5
:10087600757401F0900B907462F0A37411F0A37478
:1008860060F0A37401F0A37495F0A3743DF0A37413
:1008960090F0A37404F0A37497F0A37426F0A374E5
:1008A60093F0A37418F0A37462F0A37410F0A37409
:1008B60070F0A37430F09006817401F0900D1074FE
:1008C60062F0A37411F0A37460F0A37401F0A37432
:1008D60092F0A3744BF0A37490F0A37404F0A37485
:1008E60094F0A37438F07499A3F0A3F0A37460F0A5
:1008F600A37401F0A37462F0A37410F01222F8122C
:1009060070BED26B7F01125A967D2F7F07127793A6
:100916007D0C7F031277937D327F061277937D1EBF
:100926007F0512779390001F7401F0FD7F1F7E00F4
:0B0936001273C4C26B7F01125A96229C
:1022F8009001007402F0A3740DF0A37402F090062C
:10230800A014F09010F07464F0A37411F0A3749703
:10231800F0A3742EF0A37495F0A3743DF0A3749009
:10232800F0A37402F0A37496F0A37438F0A3746455
:10233800F0A37410F0A37470F0A37411F090010866
:102348007402F0A3740EF0A37402F09006A114F0C6
:102358009011107461F0A37410F0A37464F0A37466
:1023680011F0A37497F0A3742EF0A37495F0A374DE
:102378003DF0A37490F0A37402F0A37496F0A374D4
:1023880036F0A37464F0A37410F0A37470F0A3740F
:1023980010F09001107402F0A3740DF0A37403F010
:1023A8009006A27401F09011307464F0A37411F0D7
:1023B800A37497F0A3742EF0A37495F0A3743DF062
:1023C800A37490F0A37403F0A37496F0A37438F088
:1023D800A37464F0A37410F0A37470F0A37421F0D4
:1023E8009001187402F0A3740EF0A37403F0900621
:1023F800A37401F09011507461F0A37410F0A374E9
:1024080064F0A37411F0A37497F0A3742EF0A3746E
:1024180095F0A3743DF0A37490F0A37403F0A37433
:1024280096F0A37436F0A37464F0A37410F0A37448
:1024380070F0A37420F09001207402F0A3740DF0E2
:10244800A37404F09006A47401F09011707464F001
:10245800A37411F0A37497F0A3742EF0A37495F0ED
:10246800A3743DF0A37490F0A37404F0A37496F0E1
:10247800A37438F0A37464F0A37410F0A37470F01C
:10248800A37431F09001287402F0A3740EF0A374C1
:1024980004F09006A57401F09011907461F0A37493
:1024A80010F0A37464F0A37411F0A37497F0A374EC
:1024B8002EF0A37495F0A3743DF0A37490F0A37468
:1024C80004F0A37496F0A37436F0A37464F0A374B4
:1024D80010F0A37470F0A37430F09001307403F01E
:1024E800A3740DF0A37402F0A304F09006A674017F
:1024F800F09011B07464F0A37411F0A37497F0A372
:10250800742EF0A37495F0A3743DF0A37490F0A317
:102518007402F0A37490F0A37403F0A37496F0A36C
:102528007438F0A37464F0A37410F0A37470F0A36B
:102538007441F09001387403F0A3740EF0A3740290
:10254800F0A304F09006A77401F09011D07461F024
:10255800A37410F0A37464F0A37411F0A37497F03B
:10256800A3742EF0A37495F0A3743DF0A37490F0B7
:10257800A37402F0A37490F0A37403F0A37496F00C
:10258800A37436F0A37464F0A37410F0A37470F00D
:10259800A37440F09001407404F0A3740DF0A37488
:1025A80002F0A304F0A304F09006A87401F09011BF
:1025B800F07464F0A37411F0A37497F0A3742EF070
:1025C800A37495F0A3743DF0A37490F0A37402F083
:1025D800A37490F0A37403F0A37490F0A37404F0B0
:1025E800A37496F0A37438F0A37464F0A37410F085
:1025F800A37470F0A37441F0A37470F0A37451F045
:102608009001487404F0A3740EF0A37402F0A304BC
:10261800F0A304F09006A97401F09012107461F010
:10262800A37410F0A37464F0A37411F0A37497F06A
:10263800A3742EF0A37495F0A3743DF0A37490F0E6
:10264800A37402F0A37490F0A37403F0A37490F041
:10265800A37404F0A37496F0A37436F0A37464F022
:10266800A37410F0A37470F0A37440F0A37470F016
:05267800A37450F022E4
:0A7343008E4C8F4D8C4E8D4F8B50F9
:10734D00E4F9C3E5506480F8E96480985028E9FFBA
:10735D003395E0FEE54D2FF582E54C3EF583E49344
:10736D00FFE9FD3395E0FCE54F2DF582E54E3CF54B
:06737D0083EFF00980CC53
:0173830022E7
:107AEF00D291C2A4C2A5C2A6C2A7007F05127B670E
:097AFF0000127B5100D2A7D291C4
:017B0800225A
:107A0C00127AEFEF20E0F9D291C2A4C2A5C2A6C2AD
:0E7A1C00A7007F06127B670000D2A7D291223E
:107A2A00127AEFEF20E0F9D291C2A4C2A5C2A6C28F
:0E7A3A00A7007F04127B670000D2A7D2912222
:046EDD008E528F53EF
:106EE100AE04AF058E568F57D291C2A4C2A5C2A6D9
:106EF100C2A7007F03127B67E552FF127B67AF5386
:106F0100127B67E4F554F555127B51E5572555F58C
:106F110082E5563554F583EFF00555E555700205C8
:0E6F210054C39420E554940040DED2A7D291D0
:016F2F00223F
:086954008E5D8F5E8C5F8D608B
:10695C00127AEFEF20E0F9127A0C855D63855E64A4
:10696C00D291C2A4C2A5C2A6C2A7007F02127B67A5
:10697C00E55FFF127B67AF60127B67E4F561F56240
:10698C00E5642562F582E5633561F583E0FF127BF2
:10699C00670562E56270020561C39420E5619400AD
:0769AC0040DE00D2A7D291EA
:0169B30022C1
:0A6816008E4C8F4D8C4E8D4F8B5031
:10682000C2AF127A0C127AEFEF20E0F9854E528552
:106830004F53D291C2A4C2A5C2A6C2A7007F021222
:106840007B67E54CFF127B67AF4D127B67E4F55128
:10685000AF50EF3395E0FEC3E5519FEE6480F874CE
:1068600080985014E5532551F582E43552F583E0C4
:10687000FF127B67055180D800D2A7D291127A2AE5
:02688000D2AF95
:0168820022F3
:1073C4008E5B8F5C8D5DC2AF127A0C127AEFEF2068
:1073D400E0F9D291C2A4C2A5C2A6C2A7007F02123C
:1073E4007B67E55BFF127B67AF5C127B67AF5D1267
:0E73F4007B670000D2A7D291127A2AD2AF2274
:0478D6008E4C8F4DF8
:1078DA00D291C2A4C2A5C2A6C2A77F03127B67E542
:1078EA004CFF127B67AF4D127B67127B51D2A7D236
:0178FA0091FC
:0178FB00226A
:10722E00C2AF754E00754F20755000755120E4F5B4
:10723E004CF54DAD4FAC4EAF51AE50126EDD7420CD
:10724E00254FF54FE4354EF54E74202551F551E49A
:10725E003550F550054DE54D7002054CC394D6E5FD
:07726E004C940040CED2AFAA
:0172750022F6
:1070BE00C2AF755B00755C20755900755A20E4F5FA
:1070CE0057F558AD5AAC59AF5CAE5B12695474208B
:1070DE00255AF55AE43559F5597420255CF55CE4CA
:1070EE00355BF55B0558E55870020557C394D6E538
:0A70FE0057940040CE127A2AD2AF58
:017108002264
:046F82008C4D8D4E57
:106F8600EF6048D22BD22CD22DD22EE4F54F854E6F
:106F960082854D83E0FEA3E04E6028AF4FEF339528
:106FA600E0FEEF25E0FFEE33FEE54E2FF582E54DE0
:106FB600125544926720670B054FC3E54F648094D2
:0B6FC6009040CBC22BC22CC22DC22E6B
:016FD100229D
:047384008C4D8D4E51
:10738800EF6038E4F54F854E82854D83E0FEA3E03B
:107398004E6028AF4FEF3395E0FEEF25E0FFEE3368
:1073A800FEE54E2FF582E54D125544926720670B96
:0B73B800054FC3E54F6480949040CB6C
:0173C30022A7
:085544003EF583E0FEA3E0FF49
:04554C00AD07AC06F5
:10555000C268780CEF088006A2E0CE13CE13D8F80C
:10556000540FF5507808AF05AE04EF088006A2E0AE
:10557000CE13CE13D8F8540FF5517804AF05AE040E
:10558000EF088006A2E0CE13CE13D8F8540FF552E0
:10559000ED540FF553E550607CB4010BAB53AD52A5
:1055A000AF5112586B806EE550B4030BAB53AD5244
:1055B000AF51126ACF805EE550B4040BAB53AD52CD
:1055C000AF51126B2A804EE550B4050BAB53AD5270
:1055D000AF51123CEC803EE550B4060BAB53AD52DC
:1055E000AF5112180F802EE550B4070BAB53AD52DC
:1055F000AF51124106801EE550B4080BAB53AD52BB
:10560000AF51126F30800EE550B40909AB53AD5263
:07561000AF51127921A268DD
:015617002270
:10586B008F548D558B56E554B40113900020E0FFF7
:10587B00126A77900020EFF0FD7F20025906E55465
:10588B00B40211900021126A71900021EFF0FD7F9C
:10589B0021025906E554B40310900022126A71904C
:1058AB000022EFF0FD7F228052E554B404109000EB
:1058BB0023126A71900023EFF0FD7F23803DE554A6
:1058CB00B40510900024126A71900024EFF0FD7F54
:1058DB00248028E554B40610900025126A719000BC
:1058EB0025EFF0FD7F258013E554B40713900026B8
:1058FB00126A71900026EFF0FD7F267E000273C4C2
:10590B00E554B40816900027126A71900027EFF047
:0C591B00FD7F277E001273C412770F225C
:066A7100E0FFAB56AD553D
:106A7700D269AC07BD01047E018033BD02047E02EA
:106A8700802CBD03047E048025BD04047E08801E7F
:106A9700BD05047E108017BD06047E208010BD074B
:106AA700047E408009BD08047E808002C269BB0164
:106AB70005EE4204800BEB7006EEF452048002C22E
:076AC70069306903AF0422EE
:016ACE0022A5
:106ACF008F548D558B56E554700BAD56AF55127BC9
:106ADF00F9E4FD801EE554B4010BAD56AF55127BA2
:106AEF00F97D01800EE554B4020CAD56AF55127B03
:106AFF00F97D02023861E554B4030AE555700612B8
:106B0F007301C25822E554B40410AD56AF55126745
:0B6B1F00738F3F753D05E53D70FC22C3
:106B2A008F548D558B56E5547036E555B40108E5FA
:106B3A005614FF7D018026E555B40208E55614FF78
:106B4A007D028019E555B40308E55614FF7D0380DC
:106B5A000CE55564047022E55614FF7D0402727632
:106B6A00E554B40114E555D39400400DE555940558
:0A6B7A005007753D01E53D70FC2257
:103CEC008B54EF7017BD0114E5547002C220E554DB
:103CFC0064016003023E58D220023E58EF7017BD9B
:103D0C000214E5547002C221E55464016003023EC2
:103D1C0058D221023E58EF7017BD0314E5547002BF
:103D2C00C222E55464016003023E58D222023E587E
:103D3C00EF7017BD0414E5547002C223E5546401FE
:103D4C006003023E58D223023E58EF701BBD05188B
:103D5C00E5547004C220C221E55464016003023EA4
:103D6C0058D220D221023E58EF701BBD0618E554E4
:103D7C007004C222C223E55464016003023E58D28F
:103D8C0022D223023E58BF0117BD0114E554700224
:103D9C00C224E55464016003023E58D224023E580A
:103DAC00BF0117BD0214E5547002C225E55464012D
:103DBC006003023E58D225023E58BF0116BD0313C4
:103DCC00E5547002C226E55464016003023E58D2E9
:103DDC00268079BF0113BD0410E5547002C227E59B
:103DEC005464017067D2278063BF0117BD0514E5C9
:103DFC00547004C224C225E5546401704FD224D2FD
:103E0C00258049BF0117BD0614E5547004C226C2B3
:103E1C0027E55464017035D226D227802FEF640138
:103E2C00702AED64097025E554B401047F018019F2
:103E3C00E554B402047F028010E554B403047F03FC
:103E4C008007E554B404057F04126C377F327E0082
:043E5C00127ABA22FA
:10180F008F548D558B56E5547016AD56AF55127BD0
:10181F00F9901D14EFF0901D14E0D3940050F722AF
:10182F00E554B40117E555B40112E5567002C2082C
:10183F00E55664016003021BB5D20822E554B401DA
:10184F0017E555B40212E5567002C209E556640158
:10185F006003021BB5D20922E554B40117E555B454
:10186F000312E5567002C20EE55664016003021BB7
:10187F00B5D20E22E554B40117E555B40412E5565E
:10188F007002C20CE55664016003021BB5D20C2234
:10189F00E554B4011BE555B40516E5567004C208AE
:1018AF00C209E55664016003021BB5D208D20922B2
:1018BF00E554B40118E555B40613E5567004C20E8D
:1018CF00C20CE55664016003021BB58024E5546425
:1018DF00017023E555B4071EE5567008C208C2090A
:1018EF00C20EC20CE55664016003021BB5D208D2CA
:1018FF0009D20ED20C22E554B4021DE555B40118DD
:10190F00E5567004C208C220E55664016003021B4D
:10191F00B5D208D220021AD5E554B4021DE555B44C
:10192F000218E5567004C209C221E556640160032E
:10193F00021BB5D209D221021A61E554B4021DE58A
:10194F0055B40318E5567004C20EC222E556640161
:10195F006003021BB5D20ED222021A85E554B402DF
:10196F001DE555B40418E5567004C20CC223E556A4
:10197F0064016003021BB5D20CD223021AA8E554EE
:10198F0064027026E55564057020E5567008C2089C
:10199F00C209C220C221E55664016003021BB5D201
:1019AF0008D209D220D221021AD5E554640270263A
:1019BF00E55564067020E5567008C20EC20CC222AF
:1019CF00C223E55664016003021BB5D20ED20CD2BE
:1019DF0022D223021A85E55464027035E555640757
:1019EF00702FE5567010C208C209C20EC20CC22079
:1019FF00C221C222C223E55664016003021BB5D285
:101A0F0008D209D20ED20CD220D221D222D22380D8
:101A1F0065E554B4031DE555B40118E5567004C2CD
:101A2F0008C224E55664016003021BB5D208D22414
:101A3F00021AD5E554B4031FE555B4021AE55670E2
:101A4F0004C209C225E55664016003021BB5D20921
:101A5F00D2257F02021B04E554B4031EE555B403DF
:101A6F0019E5567004C20EC226E5566401600302E2
:101A7F001BB5D20ED2267F03807BE554B4031EE53F
:101A8F0055B40419E5567004C20CC227E55664011B
:101A9F006003021BB5D20CD2277F048058E5546433
:101AAF00037027E55564057021E5567008C208C21A
:101ABF0009C224C225E55664016003021BB5D20892
:101ACF00D209D224D2257F01802BE55464037028DC
:101ADF00E55564067022E5567008C20EC20CC22688
:101AEF00C227E55664016003021BB5D20ED20CD299
:101AFF0026D2277F03026C37E554B4040AE555B4A8
:101B0F000105AF560266B2E554B4040AE555B402B6
:101B1F0005AF560268ECE5546409701EE555B40133
:101B2F0019E5567003C20A22E556B40103D20A2200
:101B3F00E556640270707F058069E5546409701E74
:101B4F00E555B40219E5567003C20B22E556B401F0
:101B5F0003D20B22E5566402704C7F068045E55494
:101B6F006409701EE555B40319E5567003C20F22C0
:101B7F00E556B40103D20F22E556640270287F07A1
:101B8F008021E5546409701EE555B40419E55670BB
:101B9F0003C20D22E556B40103D20D22E556B4025D
:071BAF00057F081260F4221B
:104106008F548D558B56E554700FE555700BE5565B
:10411600B40306127071024214E55460030241FCB6
:10412600E555B4010DE556700990001FE054FDF009
:104136008011E555B4010CE556B4010790001FE067
:104146004403F0E555B4020DE556700990001FE0F2
:1041560054FBF08011E555B4020CE556B401079006
:10416600001FE04405F0E555B4030DE556700990CF
:10417600001FE054F7F08011E555B4030CE556B482
:10418600010790001FE04409F0E555B4040DE5561B
:10419600700990001FE054F9F08011E555B4040C45
:1041A600E556B4010790001FE04407F0E555B40555
:1041B6000DE556700990001FE054F3F08011E555A7
:1041C600B4050CE556B4010790001FE0440DF0E578
:1041D60055B4060DE556700990001FE054F1F080C5
:1041E6002DE55564067027E5566401702190001F81
:1041F600E0440FF08018E554B40113E555700FE55F
:10420600567004C2298007E556B40102D2299000EF
:0B4216001FE0FD7F1F7E001273C4221A
:106F30008F548D558B56E554700C127BF5744F2F82
:106F4000F58274068020E554B4010C127BF5744F71
:106F50002FF58274068024E554B40210127BF57478
:106F60009F2FF58274063EF583E4F022E554B403C6
:106F700010127BF5749F2FF58274063EF583740121
:026F8000F022FD
:027921008F5481
:10792300AF057804EF08800123D8FD4BF555E554E6
:10793300B40908E555B4990302605EAD55AF54121E
:02794300779338
:01794500221F
:1066B200E545B40109BF0106D220D2088060E54554
:1066C200B40109EF7006C220C2088052E545B40247
:1066D20009BF0106D221D2098044E545B40209EF7F
:1066E2007006C221C2098036E545B40309BF01061E
:1066F200D222D20E8028E545B40309EF7006C222E9
:10670200C20E801AE545B40409BF0106D223D20C99
:10671200800CE545B40407EF7004C223C20C127A60
:0A6722009EAF3E126C37127A8222FD
:1068EC00E545B40108BF0105D224D20822E545B420
:1068FC000108EF7005C224C20822E545B40208BFA6
:10690C000105D225D20922E545B40208EF7005C273
:10691C0025C20922E545B40308BF0105D226D20ED3
:10692C0022E545B40308EF7005C226C20E22E545E8
:10693C00B40408BF0105D227D20C22E545B40407E4
:08694C00EF7004C227C20C2207
:10707100D26BAF45125A96127A9E90001FE030E013
:10708100077D01E4FF12779390001FE030E1077D57
:1070910002E4FF12779390001FE030E2077D03E4E2
:1070A100FF12779390001FE030E3077D04E4FF12A5
:0D70B1007793C26BAF45125A96127A9E2259
:047BF500AD56AF5585
:0D7BF900EF75F00AA47C002DFFEC35F0FEC6
:017C0600225B
:020941008F4DD8
:10094300C268E4F53DD25ED26B125A967D4B7F02AC
:100953001277937D04E4FF1277937D387F04127737
:10096300937D607F0212779390061CE0FFA3E090D3
:100973001CE8CFF0A3EFF0C26BAF4D125A96E4F52B
:1009830046C208123346E54DB40106A24992678078
:100993001FE54DB40206A24D92678014E54DB403E2
:1009A30006A25192678009E54DB40404A2549267EC
:1009B300901CE8E07002A3E07005D268020F8B3050
:1009C30067C1123346E54DB40106A2499267801F01
:1009D300E54DB40206A24D92678014E54DB40306BB
:1009E300A25192678009E54DB40404A25492672092
:1009F30067D0E54DB4010A754E1B754F10786880BA
:100A03002BE54DB4020A754E1B754F607869801C47
:100A1300E54DB4030A754E1B754FB0786A800DE53A
:100A23004DB4040B754E1C754F00786BE6F550E51D
:100A330050D394005003020F85854F82854E83E087
:100A4300640B6003020F80A3E0FFB40A0AE550B40D
:100A53000205D268020F85EF64017032854F8285EB
:100A63004E83A3A3E064037025E550B40520854FAE
:100A730082854E83A3A3A3E0FFE54F2404F582E41C
:100A8300354EF583E0FDAB4D123FBA020F85854F1E
:100A930082854E83A3E0B40121854F82854E83A3D3
:100AA300A3E0B40415E550D39405400EAB4DAD4F10
:100AB300AC4EAF50123510020F85854F82854E83A1
:100AC300A3E064017032854F82854E83A3A3E06463
:100AD300057025E550B40520854F82854E83A3A379
:100AE300A3E0FFE54F2404F582E4354EF583E0FDF2
:100AF300AB4D1265B6020F85854F82854E83A3E009
:100B030064017032854F82854E83A3A3E06406702F
:100B130025E550B40520854F82854E83A3A3A3E02A
:100B2300FFE54F2404F582E4354EF583E0FDAB4D3C
:100B3300125CA5020F85854F82854E83A3E0B40125
:100B430021854F82854E83A3A3E0B40715E550D3D7
:100B53009405400EAB4DAD4FAC4EAF50124EC60296
:100B63000F85854F82854E83A3E064017032854FE4
:100B730082854E83A3A3E064087025E550B4052065
:100B8300854F82854E83A3A3A3E0FFE54F2404F59D
:100B930082E4354EF583E0FDAB4D126B84020F8585
:100BA300854F82854E83A3E0B40219854F82854E1B
:100BB30083A3A3E0B4080DE550B40308AF4D127747
:100BC30067020F85854F82854E83A3E064027024FC
:100BD300854F82854E83A3A3E0B40818E550B4047F
:100BE30013854F82854E83A3A3A3E0FFAD4D1278F7
:100BF30060020F85854F82854E83A3E0B402198579
:100C03004F82854E83A3A3E0B4090DE550B40308D6
:100C1300AF4D12773B020F85854F82854E83A3E04C
:100C230064027024854F82854E83A3A3E0B4091820
:100C3300E550B40413854F82854E83A3A3A3E0FF3D
:100C4300AD4D127838020F85854F82854E83A3E020
:100C530064037036854F82854E83A3A3E0640A70D4
:100C630029E55064057023854F82854E83A3A3A392
:100C7300E0FFE54F2404F582E4354EF583E0FD12F1
:100C83007A53AD4D1257AC020F85854F82854E8343
:100C9300A3E06403703E854F82854E83A3A3E06483
:100CA300017031E550D39405402A854F82854E83E8
:100CB300A3A3A3E0FFE54F2404F582E4354EF583B7
:100CC300E0FD127A53854D55AB50AD4FAC4E1247F4
:100CD30089020F85854F82854E83A3E064037036B6
:100CE300854F82854E83A3A3E064027029E5506497
:100CF300057023854F82854E83A3A3A3E0FFE54FB1
:100D03002404F582E4354EF583E0FD127A53AD4DAC
:100D1300127154020F85854F82854E83A3E0B4037D
:100D230019854F82854E83A3A3E0B4030DE550B428
:100D33000308AF4D127402020F85854F82854E83DF
:100D4300A3E0B40321854F82854E83A3A3E0B404BB
:100D530015E550D39403400EAB4DAD50AF4FAE4E9F
:100D6300125F2D020F85854F82854E83A3E0B40366
:100D730019854F82854E83A3A3E0B4050DE550B4D6
:100D83000308AF4D127C07020F85854F82854E8382
:100D9300A3E0B4031D854F82854E83A3A3E0B4066D
:100DA30011E550B4050CAD4DAF4FAE4E12747B023E
:100DB3000F85854F82854E83A3E064037024854F9E
:100DC30082854E83A3A3E0B40718E550B4041385CA
:100DD3004F82854E83A3A3A3E0FFAD4D1279CD02CD
:100DE3000F85854F82854E83A3E0B4031D854F8213
:100DF300854E83A3A3E0B40811E550B4050CAD4DB3
:100E0300AF4FAE4E127655020F85854F82854E83C6
:100E1300A3E064057022E550B4041D854F82854E1E
:100E230083A3A3E0FF854F82854E83A3A3A3E0FDA5
:100E3300AB4D122D80020F85854F82854E83A3E033
:100E4300B40524E54F2404F582E4354EF583E0B47C
:100E53000B15E550D39405400EAB4DAD50AF4FAEDF
:100E63004E124899020F85854F82854E83A3E06415
:100E7300067022E550B4041D854F82854E83A3A3DB
:100E8300E0FF854F82854E83A3A3A3E0FDAB4D1204
:100E9300267D020F85854F82854E83A3E0B4062409
:100EA300E54F2404F582E4354EF583E0B40B15E5F4
:100EB30050D39405400EAB4DAD50AF4FAE4E1231F3
:100EC3005E020F85854F82854E83A3E064097022FD
:100ED300854F82854E83A3A3E0B40A16E550B4047C
:100EE30011854F82854E83A3A3A3E0FF12710902EC
:100EF3000F85854F82854E83A3E064097023854F58
:100F030082854E83A3A3E0B40117E550B404128590
:100F13004F82854E83A3A3A3E0FFAD4D1256E88015
:100F230061854F82854E83A3E0B40920854F828576
:100F33004E83A3A3E0B40214E550D39404400DAB55
:100F430050AD4DAF4FAE4E1214648036854F82853F
:100F53004E83A3E064097025854F82854E83A3A346
:100F6300E0B40317E550B40412854F82854E83A382
:100F7300A3A3E0FFAD4D126FD280078000AF4D12E7
:100F83007A65206803020986C258D26BAF4D125AA4
:100F9300967D607F021277937D327F03127793C22F
:0F0FA3006BAF4D125A961270BEE4786CF6C25EB8
:010FB200221C
:083510008F518C528D538B5436
:10351800855382855283A3A3A3E0FF8D828C83E524
:1035280082240412676A8F55E555D394005003022C
:1035380036B1E555942940030236B1E55164067069
:103548004FD26BAF54125A967D527F05127793AFC4
:1035580055124CC4E5532405F582E43552F583E051
:10356800B40112749F2555F582E43406F58374017D
:10357800F07D38800F749F2555F582E43406F58375
:10358800E4F07D367F06127793C26BAF54025A96E9
:10359800E5532406F582E43552F583E0640B6003B5
:1035A8000236B1E5532405F582E43552F583E0B4DB
:1035B8000110749F2555F582E43406F5837401F0F3
:1035C800800D749F2555F582E43406F583E4F0E414
:1035D800FFFEE5532407F582E43552F583E5822E94
:1035E800F582E43583F583E0B40B04AF0680040E5E
:1035F800BE08DFEF70030236B1C3940840030236F9
:10360800B175F008E555A424F8F582E5F03400F525
:1036180083EFF07E01EF2401FDE433FCEEC39DEC63
:103628006480F87480985036E5532406F582E435B2
:1036380052F583E5822EF582E43583F583E0FD7546
:10364800F008E555A424F8F582E5F03400F583E5A3
:10365800822EF582E43583F583EDF00E80B7E553CD
:103668002408F582E43552F583E5822FF582E435A6
:1036780083F583E0640B602DEF2408FEC3E5519EBB
:10368800F55175F004125927AEF0EE701CE553247D
:1036980007FDE43552FC7E00ED2FFBEE3CFAAD55FC
:1036A8007F011239EAD26A8002C26AAF54127C39A9
:0136B80022EF
:10796A008E5CF55DAF5BEF3395E0FEE5592FF5824E
:08797A00E5583EF583A3E0FF90
:0A798200EFD3940940037F00222296
:0839EA008F568D578A588B5946
:1039F200755B01E4F55AAF5BEF3395E0FEE5592FB5
:103A0200F582E5583EF583E0FF640970651279821C
:103A1200755C008F5DAE5C7804EF08800633CE33B0
:103A2200CE92E0D8F812796AEF425DAE5CAF5D7873
:103A320008EF08800633CE33CE92E0D8F88E5CF5DC
:103A42005DAF5BEF3395E0FEE5592FF582E5583E19
:103A5200F583A3A3E0FFE55BFD3395E0FCE5592D7B
:103A6200F582E5583CF583A3A3A3E0FD127A530245
:103A72003B05AF5BEF3395E0FEE5592FF582E55844
:103A82003EF583E0FF127982755C008F5DAE5C7853
:103A920004EF08800633CE33CE92E0D8F812796A6A
:103AA200EF425DAE5CAF5D7804EF08800633CE3343
:103AB200CE92E0D8F88E5CF55DAF5BEF3395E0FE19
:103AC200E5592FF582E5583EF583A3A3E0FF12796D
:103AD20082EF425DAE5CAF5D7804EF08800633CEC4
:103AE20033CE92E0D8F88E5CF55DAF5BEF3395E0B4
:103AF200FEE5592FF582E5583EF583A3A3A3E0FF27
:103B0200127982EF425DE556701EAF5AEF3395E0AF
:103B1200FEEF25E0FFEE33FE75F020E557A424D03A
:103B2200F582E5F034068021E556B4012FAF5AEF55
:103B32003395E0FEEF25E0FFEE33FE75F020E5570A
:103B4200A424D0F582E5F03410F583E5822FF582C6
:103B5200E5833EF583E55CF0A3E55DF07404255B47
:103B6200F55B055AC3E55A6480949050030239F814
:013B72002230
:084EC6008F518C528D538B5467
:104ECE00855382855283A3A3A3E0FF8D828C83E555
:104EDE0082240412676A8F55E555D394005003025D
:104EEE004FB3E55594334003024FB3E5516406705A
:104EFE004FD26BAF54125A967D527F05127793AFF5
:104F0E0055124CC4E5532405F582E43552F583E081
:104F1E00B40112744F2555F582E43406F5837401FD
:104F2E00F07D38800F744F2555F582E43406F583F5
:104F3E00E4F07D367F06127793C26BAF54025A9619
:104F4E00E5532406F582E43552F583E0640B705583
:104F5E00E5532405F582E43552F583E0B40110746F
:104F6E004F2555F582E43406F5837401F0800D74F7
:104F7E004F2555F582E43406F583E4F074F9255196
:104F8E00F55175F004125927AFF0EF7014E5532464
:104F9E0006FBE43552FAAD55E4FF1239EAD26A80C7
:104FAE000DC26A8009C26BAF54125A96C26AAF54D0
:034FBE00127C3929
:014FC10022CD
:023FBA008B5129
:103FBC001267738F54E554D3940050030240FEE50E
:103FCC0054943340030240FED26BAF51125A967D8B
:103FDC00527F05127793AF54124CC4749F2554F53D
:103FEC0082E43406F583E060047D3880027D367F00
:103FFC00061277937F2C7E01127ABA75F008E5547D
:10400C00A424F8F582E5F03400F583E0F55270074E
:10401C007D1B7F061277937D577F02127793E552B3
:10402C0070030240AF755301AF52EF3395E0FEEFD2
:10403C002401FFE43EFEAD53ED3395E0FCC3ED9F50
:10404C00EE6480F8EC6480985059AF53EF3395E0F0
:10405C00FE75F008E554A424F8F582E5F03400F57B
:10406C0083E5822FF582E5833EF583E0FFD3940947
:10407C0040051272BC8028AF53EF3395E0FE75F00B
:10408C0008E554A424F8F582E5F03400F583E582C4
:10409C002FF582E5833EF583E0FDE4FF127793056F
:1040AC005380857F2C7E01127ABA75F020E554A4DA
:1040BC0024D0F582E5F03410F583E0FEA3E0FF9008
:1040CC000000EEF0A3EFF04E70077D1B7F06127719
:1040DC00937D0C7F03127793900000E07002A3E0B5
:1040EC006009E55414FD7F01122F74C26BAF5102AD
:0940FC005A96C26AAF51127C39D8
:014105002297
:042F74008F558D5692
:102F7800E4F557E555600302301FAF57EF3395E08E
:102F8800FEEF25E0FDEE33FCAF56EF3395E0FEEFA4
:102F98007805C333CE33CED8F924F0F58274063ED3
:102FA800F583E5822DF582E5833CF583E0FAA3E01D
:102FB800FB780CFFAE02088006A2E0CE13CE13D831
:102FC800F8540FF5587808AF03AE02EF088006A250
:102FD800E0CE13CE13D8F8540FF559AF56EF33950A
:102FE800E0FEEF7805C333CE33CED8F924F0F5826E
:102FF80074063EF583E5822DF582E5833CF583E092
:10300800FCA3E0FD7804FFAE04088006A2E0CE131E
:10301800CE13D8F80230C2E555640160030230CB04
:10302800AF57EF3395E0FEEF25E0FDEE33FCAF56EA
:10303800EF3395E0FEEF7805C333CE33CED8F924CD
:10304800F0F58274103EF583E5822DF582E5833C28
:10305800F583E0FAA3E0FB780CFFAE02088006A235
:10306800E0CE13CE13D8F8540FF5587808AF03AE56
:1030780002EF088006A2E0CE13CE13D8F8540FF55D
:1030880059AF56EF3395E0FEEF7805C333CE33CE14
:10309800D8F924F0F58274103EF583E5822DF58287
:1030A800E5833CF583E0FCA3E0FD7804FFAE04086B
:1030B8008006A2E0CE13CE13D8F8540FF55AED547B
:1030C8000FF55BE558700FE559700BE55A7007E589
:1030D8005B700302315DAD58E4FF127793AD59E49C
:1030E800FF127793E55864097048855A5CAF5CFE17
:1030F8007804EF08800633CE33CE92E0D8F8F55C3A
:10310800E55B425CE55CB4990B7D09E4FF127793BB
:103118007D098027E55C75F00A84F55DFDE4FF1202
:103128007793E55D75F00AA4FFC3E55C9FF55DFD47
:103138008009AD5AE4FF127793AD5BE4FF127793F1
:103148007FF47E01127ABA0557C3E557648094A0CC
:053158005003022F7B73
:01315D00224F
:025CA5008B5121
:105CA7001267738F52E552D394005003025D41E5AA
:105CB7005294334003025D41D26BAF51125A967D25
:105CC700527F05127793AF52124CC4744F2552F589
:105CD70082E43406F583E060047D3880027D367FF8
:105CE700061277937F2C7E01127ABA7F2C7E0112DF
:105CF7007ABA75F020E552A424D0F582E5F034068F
:105D0700F583E0FEA3E0FF900000EEF0A3EFF04E76
:105D170070077D1B7F061277937D0C7F03127793A5
:105D2700900000E07002A3E06009E55214FDE4FF73
:105D3700122F74C26BAF51025A96C26AAF51127CCE
:015D47003922
:015D48002238
:0265B6008B5107
:1065B800126773AD07EDD39400406BED94335066CA
:1065C800E4FCECFF3395E0FEEF25E0FFEE33FE75CB
:1065D800F020EDA424D0F582E5F03410F583E582AF
:1065E8002FF582E5833EF583E4F0A3F00CBC10D2CE
:1065F800749F2DF582E43406F583E4F0FCECFF3358
:1066080095E0FE75F008EDA424F8F582E5F0340075
:10661800F583E5822FF582E5833EF583E4F00CBC33
:0D66280008DBD26A8002C26AAF51127C39D1
:016635002242
:026B84008B5133
:106B8600126773AD07EDD394004045ED9433504042
:106B9600E4FCECFF3395E0FEEF25E0FFEE33FE75F7
:106BA600F020EDA424D0F582E5F03406F583E582E5
:106BB6002FF582E5833EF583E4F0A3F00CBC10D2FA
:106BC600744F2DF582E43406F583E4F0D26A800230
:076BD600C26AAF51127C39C5
:016BDD002295
:1075F0002430F58274003EF583EDF0AF55EF3395FE
:10760000E0FEE5522FF582E5513EF583A3A3E0FFAE
:10761000D3EF648094814008EF6480948A50012203
:037620007F0022C6
:107BE200D3EF648094804008EF648094A150012216
:037BF2007F0022EF
:081464008E518F528D538B5401
:10146C008F828E83A3A3A3E014F55674FC2554F548
:10147C00546403600FE55464076009E554640B6021
:10148C0003021807C3E556648094805003021807C2
:10149C00E556648094884003021807E4F555AF566E
:1014AC00EF3395E0FEEF7803C333CE33CED8F92477
:1014BC0030F58274003EF583AF55EF3395E0FEE5D1
:1014CC00822FF582E5833EF583E4F00555E555B4AE
:1014DC0008CC755504E5546403705FAF55EF339534
:1014EC00E0FEE5522FF582E5513EF583E0FFE55530
:1014FC00FD3395E0FCE5522DF582E5513CF583A3D7
:10150C00E0FD126773127BE2AD07AF56EF3395E047
:10151C00FEEF7803C333CE33CED8F91275F0AD0796
:10152C00AF56EF3395E0FEEF7803C333CE33CED80E
:10153C00F92431F58274000217FEE5546407600348
:10154C00021639AF55EF3395E0FEE5522FF582E5E3
:10155C00513EF583E0FFE555FD3395E0FCE5522D5A
:10156C00F582E5513CF583A3E0FD126773127BE233
:10157C00AD07AF56EF3395E0FEEF7803C333CE33B0
:10158C00CED8F91275F0AD07AF56EF3395E0FEEFFC
:10159C007803C333CE33CED8F92431F58274003EB0
:1015AC00F583EDF0AF55EF3395E0FEE5522FF58264
:1015BC00E5513EF583A312760CAD07AF56EF33958C
:1015CC00E0FEEF7803C333CE33CED8F912672C127A
:1015DC007BE2AD07AF56EF3395E0FEEF7803C333F4
:1015EC00CE33CED8F92433F58274003EF583EDF07A
:1015FC00AF55EF3395E0FEE5522FF582E5513EF500
:10160C0083E5822406F582E43583F583E0FF1276C8
:10161C0010AD07AF56EF3395E0FEEF7803C333CE32
:10162C0033CED8F92434F58274000217FEE55464E5
:10163C000B6003021807AF55EF3395E0FEE5522F10
:10164C00F582E5513EF583E0FFE555FD3395E0FC71
:10165C00E5522DF582E5513CF583A3E0FD1267734D
:10166C00127BE2AD07AF56EF3395E0FEEF7803C384
:10167C0033CE33CED8F91275F0AD07AF56EF3395A4
:10168C00E0FEEF7803C333CE33CED8F92431F582A4
:10169C0074003EF583EDF0AF55EF3395E0FEE55267
:1016AC002FF582E5513EF583A312760CAD07AF56AC
:1016BC00EF3395E0FEEF7803C333CE33CED8F91277
:1016CC00672C127BE2AD07AF56EF3395E0FEEF7857
:1016DC0003C333CE33CED8F92433F58274003EF5F0
:1016EC0083EDF0AF55EF3395E0FEE5522FF582E533
:1016FC00513EF583E5822406F582E43583F583E0DB
:10170C00FF127610AD07AF56EF3395E0FEEF78037E
:10171C00C333CE33CED8F92434F58274003EF5832E
:10172C00EDF0AF55EF3395E0FEE5522FF582E55124
:10173C003EF583E5822407F582E43583F583E0FFEB
:10174C00127610AD07AF56EF3395E0FEEF7803C37A
:10175C0033CE33CED8F92435F58274003EF583EDC3
:10176C00F0AF55EF3395E0FEE5522FF582E5513E93
:10177C00F583E5822408F582E43583F583E0FFE503
:10178C0055FD3395E0FCE5522DF582E5513CF58392
:10179C00E582240912676A127BE2AD07AF56EF337C
:1017AC0095E0FEEF7803C333CE33CED8F92436F56B
:1017BC008274003EF583EDF0AF55EF3395E0FEE516
:1017CC00522FF582E5513EF583E582240AF582E439
:1017DC003583F583E0FF127610AD07AF56EF3395E6
:1017EC00E0FEEF7803C333CE33CED8F92437F5823D
:1017FC0074003EF583EDF0D26A8002C26AAF5312D8
:02180C007C3925
:01180E0022B7
:10710900EF24FE601014601314601624037016D265
:1071190008D2248010D209D225800AD20ED2268024
:1071290004D20CD2277FF47E01127ABA753D04E5A8
:107139003D70FC7F647E00127ABAC224C225C22641
:0B714900C227C208C209C20EC20C22FD
:0456E8008D51AC072D
:1056EC00C3EC6480948150030257ABEC64809489C2
:1056FC0040030257ABE4F552AF51EF3395E0FEEFA8
:10570C007803C333CE33CED8F924E8F582741A3E2D
:10571C00F583AF52EF3395E0FEE5822FF582E583FA
:10572C003EF583E0FD74182FF582741D3EF583ED74
:10573C00F00552E552B408C0EC14FFAD511272766C
:10574C00D269AF51125B4A753D017F327E00127AED
:10575C00BAE53D70FCC269AF51125B4AE4F552E503
:10576C0052FD3395E0FC74182DF582741D3CF583C5
:10577C00E0FBAF51EF3395E0FEEF7803C333CE334C
:10578C00CED8F924E8F582741A3EF583E5822DF51E
:0F579C0082E5833CF583EBF00552E552B408C07B
:0157AB0022DB
:046FD2008D51AC072A
:106FD600D3EC64809480403CEC648094895035E422
:106FE600FDECFF3395E0FEEF7803C333CE33CED806
:106FF600F92428F58274003EF583EDFF3395E0FE13
:10700600E5822FF582E5833EF583E4F00DBD08D1D8
:0B701600D26A8002C26AAF51127C39BE
:01702100224C
:044789008C528D536E
:10478D00D3EF648094805003024891EF6480949538
:10479D004003024891EB648094875003024891EBEB
:1047AD00648094E44003024891EF3395E0FEEF7886
:1047BD0005C333CE33CED8F92460F58274033EAFF2
:1047CD0082F5568F57EB24FBF558D3940250030214
:1047DD004891E55875F00384E5F06003024891E5D2
:1047ED005875F00384F55AC394104003024891059F
:1047FD0057E557AE567002055614F5828E83E55A6D
:10480D00F074052553F553E43552F552E4F558E5AA
:10481D0058C3955A506A855382855283E0F559B431
:10482D000A130557E557AE567002055614F5828EDC
:10483D0083E4F080120557E557AE56700205561405
:10484D00F5828E83E559F0855382855283A3E0FF6F
:10485D00855382855283A3A3E0FD127A538F5905A8
:10486D0057E557AE567002055614F5828E83E559FD
:10487D00F074032553F553E43552F5520558808FE6
:0B488D00D26A8002C26AAF55127C396B
:0148980022FD
:0457AC008F518D523A
:1057B000E551D394005003025863E551941540031A
:1057C000025863D26BAF52125A967D5F7F051277F3
:1057D00093AD51E4FF1277937D527F041277937F4C
:1057E000F47E01127ABA75F020E551A42460F582A6
:1057F000E5F03403AF82F5558F56F583E0F553603D
:105800004DD394004056E55394105050E55325E095
:10581000F553755401E5532401FFE433FEC3E55409
:105820009FEE6480F87480985032E5562554F582D6
:10583000E43555F583E0FFE5562554F582E435550A
:10584000F583A3E0FD1277930554055480C77D1BB3
:105850007F061277937D5F7F05127793C26BAF52FD
:0A586000025A96C26AAF52127C3958
:01586A00221B
:107838008D51EFD3940A4006EFD3940F4003EF70B5
:107848000E90063FEFF0D26AAF51127C39D322C2B4
:087858006AAF51127C39C32212
:107860008D51EFD3940A4006EFD3940F4003EF708D
:107870000E90063BEFF0D26AAF51127C39D322C290
:087880006AAF51127C39C322EA
:1072BC008F55E555B40B067D5F7F078034E555B4DB
:1072CC000C067D5E7F068029E555B40D067D0A7F90
:1072DC0002801EE555B40E067D327F028013E55503
:1072EC00B40F067D467F028008E55570077D0A7F46
:0572FC0003127793224C
:10773B008F51D26B125A967D207F051277937D2E37
:10774B007F031277937D527F0412779390063FE06D
:0C775B00FF1272BCC26BAF51125A962292
:107767008F51D26B125A967D207F051277937D2118
:107777007F061277937D527F0412779390063BE042
:0C778700FF1272BCC26BAF51125A962266
:1079CD008D51D3EF64809480400EEF648094865087
:1079DD0007127554D26A8002C26AAF51127C3922E5
:06747B008D51AB07AA06CB
:107481008B828A83A3A3A3E0FFEB2404F582E43A71
:1074910012676FD3EF648094804010EF648094A1F1
:1074A100500990063DEFF0D26A8002C26AAF5112D4
:0274B1007C3924
:0174B30022B6
:067655008D51AB07AA06EF
:10765B008B828A83A3A3A3E0FFEB2404F582E43A95
:10766B0012676FEFC39421500990063CEFF0D26A7A
:09767B008002C26AAF51127C3991
:0176840022E3
:065F2D008E518F528B53D0
:105F3300755406755540D3ED64809484407CED64BC
:105F43008094A55075ED24FDF556D39404406BE57C
:105F53005620E06613F5570555E555AE5470020516
:105F63005414F5828E83E557F074032552F552E4F9
:105F73003551F551E4F556E556C3955750338552DF
:105F830082855183E0FFA3E0FD127A530555E55561
:105F9300AC547002055414F5828C83EFF00552E57E
:105FA30052700205510552E55270020551055680A3
:105FB300C6D26AAF53127C39D322C26AAF53127C62
:025FC30039C3E0
:015FC50022B9
:084899008E518F528D538B5498
:1048A100C269D3E55364809484500302494EE553B1
:1048B1006480948D400302494E8F828E83A3A3E0CE
:1048C100640A600302494E8F828E83A3A3A3E0147E
:1048D100B4080050769048E475F003A4C58325F030
:1048E100C583730248FC02490602491002491A02B3
:1048F100492402492E02493802494275550075562C
:1049010080D2698048755500755688D269803E7598
:104911005500755690D2698034755500755698D2F8
:1049210069802A7555007556A0D269802075550099
:104931007556A8D26980167555007556B0D2698032
:104941000C755500755678D2698002C2693069507C
:10495100E4FFEF7C002556FDEC35558D82F583E4AF
:10496100F00FBF08EDE55324FB855682855583F092
:104971007F01E5522404F582E43551F583E5822F68
:10498100F582E43583F583E0FEEF7C002556FDECEE
:1049910035558D82F583EEF00FBF08D6D26A8002BD
:0749A100C26AAF54127C3919
:0149A80022EC
:046215008E548F55BF
:106219000555E5557002055414F5828E83E0F5574E
:106229006074C39408506F7F2C7E01127ABAE4F52A
:1062390056E556C39557505E855582855483E0606F
:106249003624F5601414601714601A14601D146064
:106259002024057028E4FD802D7D5F7F0780287D3F
:106269005E7F0680227D0A7F02801C7D327F02804C
:10627900167D467F0280107D0A7F03800A8555823C
:10628900855483E0FDE4FF1277930555E5557002C7
:0662990005540556809B30
:01629F0022DC
:022D80008B5175
:102D8200C269EF640A6003022F5BED14B4080040CD
:102D920003022F59902DA475F003A4C58325F0C515
:102DA2008373022DBC022DF0022E24022E58022E15
:102DB2008C022EC0022EF3022F26D26BAF51125A72
:102DC200967D577F021277937D05E4FF127793E495
:102DD200FDFF1277937D01E4FF1277937D527F040A
:102DE200127793755200755380D269022F5BD26BB2
:102DF200AF51125A967D577F021277937D05E4FFF9
:102E0200127793E4FDFF1277937D02E4FF1277932A
:102E12007D527F04127793755200755388D26902EE
:102E22002F5BD26BAF51125A967D577F0212779366
:102E32007D05E4FF127793E4FDFF1277937D03E4AF
:102E4200FF1277937D527F04127793755200755368
:102E520090D269022F5BD26BAF51125A967D577F87
:102E6200021277937D05E4FF127793E4FDFF127758
:102E7200937D04E4FF1277937D527F04127793755A
:102E82005200755398D269022F5BD26BAF51125A1E
:102E9200967D577F021277937D05E4FF127793E4C4
:102EA200FDFF1277937D05E4FF1277937D527F0435
:102EB2001277937552007553A0D269022F5BD26BC1
:102EC200AF51125A967D577F021277937D05E4FF28
:102ED200127793E4FDFF1277937D06E4FF12779356
:102EE2007D527F041277937552007553A8D2698080
:102EF20068D26BAF51125A967D577F021277937D3B
:102F020005E4FF127793E4FDFF1277937D07E4FF58
:102F12001277937D527F041277937552007553B0E6
:102F2200D2698035D26BAF51125A967D577F021209
:102F320077937D05E4FF127793E4FDFF1277937D8B
:102F420008E4FF1277937D527F0412779375520043
:102F5200755378D2698002C269306909AF53AE52A3
:102F62001262158005AF51127A65C26BAF51125AC7
:012F720096C8
:012F7300223B
:08315E008E518F528D538B54EA
:10316600C2698F828E83A3A3E0640A6003023215CC
:10317600124BBD8E568F57D3E557943BE5569400B8
:103186005003023210E5579408E5569407507BC366
:10319600E5536480948A5072855282855183A3A335
:1031A600A3E0F555B401069006000232BBE555B41E
:1031B60002069006020232BBE555B40306900604E9
:1031C6000232BBE555B404069006060232BBE5554D
:1031D600B405069006080232BBE555B4060690060D
:1031E6000A0232BBE555B4070690060C0232BBE56F
:1031F60055B4080690060E0232BBE555B409069092
:1032060006100232BBD269023337D26902333785E0
:103216005282855183A3A3E0640160030232C5ADE7
:1032260053AF52AE51124BBD8E568F57D3E55794BE
:103236003BE55694005003023337E5579408E556AC
:1032460094074003023337C3E5536480948A4003EE
:10325600023337855282855183A3A3A3E0F555B483
:103266000A05900612804EE555B4010590061480B5
:1032760044E555B40205900616803AE555B40305B3
:103286009006188030E555B4040590061A8026E5A8
:1032960055B4050590061C801CE555B40605900638
:1032A6001E8012E555B407059006208008E555B442
:1032B6000809900622E556F0A3806FD269807285D0
:1032C6005282855183A3A3E064027065AD53AF5269
:1032D600AE51126BDE7556008F57C3E5579463E502
:1032E600569400504CC3E5536480948850438552ED
:1032F60082855183A3A3A3E0F555B4010790063058
:10330600EFF0802DE555B40205900631801CE55599
:10331600B403059006328012E555B40405900633D1
:103326008008E555B40508900634E557F08002D2CA
:0F33360069306904C26A8002D26AAF54127C39CE
:013345002265
:10267D008F518D528B53E551640A6003022729E572
:10268D0052C3940A40030228FFD26BAF53125A96DD
:10269D007D277F081277937D06E4FF127793E4FD83
:1026AD00FF127793AD52E4FF1277937D527F0412A0
:1026BD007793E55214B4090040030228F89026D808
:1026CD0075F003A4C58325F0C583730226F3022696
:1026DD00F90226FF02270502270B022711022717F1
:1026ED0002271D02272390060002283990060202B8
:1026FD0028399006040228399006060228399006DA
:10270D000802283990060A02283990060C02283949
:10271D0090060E022839900610022839E551640101
:10272D006003022847E552D394004006E552940910
:10273D004009E552640A6003022844D26BAF53127C
:10274D005A967D277F081277937D06E4FF127793C3
:10275D00E552B40A147D0AE4FF1277937D527F048B
:10276D00127793900612022839E552B401147D0BAD
:10277D00E4FF1277937D527F041277939006140233
:10278D002839E552B402147D0CE4FF1277937D5283
:10279D007F04127793900616022839E552B403137D
:1027AD007D0DE4FF1277937D527F0412779390068F
:1027BD00188079E552B404137D0EE4FF1277937DF2
:1027CD00527F0412779390061A8061E552B4051377
:1027DD007D0FE4FF1277937D527F0412779390065D
:1027ED001C8049E552B406137D10E4FF1277937DEA
:1027FD00527F0412779390061E8031E552B4071371
:10280D007D11E4FF1277937D527F0412779390062A
:10281D00208019E552640860030229067D12FF121B
:10282D0077937D527F04127793900622E0FEA3E00A
:10283D00FF12751F0229060228FFE551640260038D
:10284D00022906E552D3940050030228FFE5529465
:10285D000740030228FFD26BAF53125A967D277F94
:10286D00081277937D06E4FF1277937D14E4FF122F
:10287D007793E55224FE602014603014604014609C
:10288D0050240470667D01E4FF1277937D527F041E
:10289D00127793900630804A7D02E4FF1277937D84
:1028AD00527F0412779390063180377D03E4FF1237
:1028BD0077937D527F0412779390063280247D04A6
:1028CD00E4FF1277937D527F041277939006338045
:1028DD00117D05E4FF1277937D527F04127793905B
:1028ED000634E0FF7E00127685800EAF53127A65B6
:1028FD008007C26AAF53127C39C26BAF53125A961E
:01290D0022A7
:064BBD008E588F59A90576
:104BC3007D057C00E5592DF582E5583CF583E0C36E
:104BD300940A400CE5592DF582E5583CF583E4F041
:104BE3000DBD00010CED640A4C70D9B90610E559EE
:104BF3002405F582E43558F583E0FF7E0022E9645D
:104C0300077019E5592405F582E43558F583E075F5
:104C1300F00AA4ACF0FDE55924068032E96408707B
:104C23003DE5592405F582E43558F583E075F064D4
:104C3300A4ACF0FDE5592406F582E43558F583E08C
:104C430075F00AA42DFDE5F03CFCE5592407F58237
:104C5300E43558F583E02DFDE43CAF05FE22E9641D
:104C630009705AE5592405F582E43558F583E0FFC8
:104C73007E007C037DE8125949AC06AD07E5592453
:104C830006F582E43558F583E075F064A42DFDE55F
:104C9300F03CFCE5592407F582E43558F583E075CB
:104CA300F00AA42DFDE5F03CFCE5592408F582E467
:104CB3003558F583E02DFDE43CFEAF0522E4FEFF0D
:014CC30022CE
:066BDE008E588F59A90535
:106BE4007F057E00E5592FF582E5583EF583E0C325
:106BF400940A400CE5592FF582E5583EF583E4F0FC
:106C04000FBF00010EEF64084E70D9E964077020CD
:106C1400E5592405F582E43558F583E075F00AA4B6
:106C2400FFE5592406F582E43558F583E02FFF2269
:026C34007F00DF
:016C3600223B
:104CC4008F56E556D3945940147D5AE4FF127793D6
:104CD400E55624A6FD7003024DC5024DC0E556D32A
:104CE400944F401AE556945A50147D50E4FF1277BD
:104CF40093E55624B0FD7003024DC5024DC0E55640
:104D0400D39445401AE556945050147D46E4FF125E
:104D14007793E55624BAFD7003024DC5024DC0E5F4
:104D240056D3943B4019E556944650137D3CE4FF1A
:104D3400127793E55624C4FD7003024DC5807DE5CA
:104D440056D394314016E556943C50107D32E4FF1E
:104D5400127793E55624CEFD60678060E556D394C0
:104D6400274016E556943250107D28E4FF127793BD
:104D7400E55624D8FD604A8043E556D3941D401679
:104D8400E556942850107D1EE4FF127793E55624CF
:104D9400E2FD602D8026E556D394134016E5569423
:104DA4001E50107D14E4FF127793E55624ECFD6049
:104DB400108009E556C394145007AD56E4FF1277EA
:024DC400932238
:107685008E548F557C007D0A12595BAD07E4FF12BD
:1076950077937D5B7F06127793AE54AF557C007D63
:1076A5000A12595BE4FF1277937D4A7F07027793AD
:04751F008E548F55A2
:107523007C007D3C12595BAA06AB07124CC47D0557
:107533007F06127793AE54AF557C007D3C12595BA6
:10754300ED4C600CAF05124CC47D4A7F0712779354
:017553002215
:027154008D515B
:10715600D3EF648094804038EF648094955031EF8B
:107166003395E0FEEF7805C333CE33CED8F92460ED
:10717600F58274033EAF82FEE4FD0FEFAA067001AE
:107186000E14F5828A83E4F00DBD20EED26A8002E9
:07719600C26AAF51127C39FF
:01719D0022CF
:107402008F51900640E0D394024015D269125B4A34
:10741200753D037F327E00127ABAE53D70FC80151D
:10742200D269AF51125B4A7D1B7F061277937D0CA6
:0D7432007F03127793C269AF51125B4A22AB
:107C07007E10900640E4F0A3DEFC7E10D26A127C60
:017C17003933
:017C18002249
:107946008F5CD26B125A967D607F021277937D32DE
:107956007F061277937D1E7F05127793C26BAF5C0D
:04796600125A9622F9
:107A65008F5CD26B125A967D607F021277937D30C0
:0D7A75007F03127793C26BAF5C125A96220A
:0E7C39008F5B306A03027946AF5B127A6522D8
:10672C002432F58274003EF583EDF0AF55EF3395CE
:10673C00E0FEE5522FF582E5513EF583E582240417
:10674C00F582E43583F583E0FFE555FD3395E0FCF8
:10675C00E5522DF582E5513CF583E5822405F58261
:07676C00E43583F583E0FD35
:10677300EFD394004015EF940B5010EFC3940A50DD
:1067830008EF75F00AA4FE8002E4FEEDD394004006
:106793000EED940B5009EDC3940A5003ED2EFEAF9A
:0167A30006EF
:0167A40022D2
:03000000027C2A55
:0F7C2A00758E0078FEE4F6D8FD75816C0252A2CB
:107B5100D292C0F075F008C29100A29233D291D5B1
:067B6100F0F5D0F0FF2258
:107B6700EFC0F075F00833C291929333D291D5F0FC
:067B7700F6D0F0C29122DD
:10779300EFFEEDFF1280008E2F8F30125D49755F73
:1077A30064AF5F155FEFD39400400EE4F55EE55ED2
:0977B300C3943A50EC055E80F528
:0177BC0022AA
:105D4900D2A885A86175A881C244853082852F8330
:105D5900E493F560C4540FF5604360F0856080C238
:105D690084D28500C2870000D287007580FF7580C4
:105D7900FEC284C28500C28700000000D287007578
:105D890080FFD24475623E756380E4F56030941DEE
:105D99000560E560B464F6123346E5631563700285
:105DA9001562D3E5639400E562940050DD75623EA7
:105DB900756380E4F56020941D0560E560B464F6C0
:105DC900123346E563156370021562D3E5639400E7
:105DD900E562940050DD8561A8C2A87F147E001297
:025DE9007ABA84
:015DEB002295
:1077BD007580FDC284C28500C28700000000D2879B
:1077CD00007580FF7F147E00127ABA7F997E0912B0
:0A77DD0080008E2F8F30125D4922CC
:10592700C2D530F707B2D563F0FF05F030E70CB208
:10593700D5F4048463F0FF05F080018430D502F4C8
:02594700042238
:10594900EF8DF0A4A8F0CF8CF0A428CE8DF0A42E72
:02595900FE222C
:10595B00BC000BBE0029EF8DF084FFADF022E4CC30
:10596B00F875F008EF2FFFEE33FEEC33FCEE9DECF9
:10597B00984005FCEE9DFE0FD5F0E9E4CEFD22ED3F
:10598B00F8F5F0EE8420D21CFEADF075F008EF2F89
:10599B00FFED33FD4007985006D5F0F222C398FD7A
:0559AB000FD5F0EA2217
:1059B000EB9FF5F0EA9E42F0E99D42F0E89C45F04D
:0159C00022C4
:1059C1007401FF3395E0FEFDFC080808E6CF2FF6D1
:1059D10018E6CE3EF618E6CD3DF618E6CC3CF622AA
:107C1900EFC39461400AEF947B5005EF24E0FF2203
:017C29002238
:00000001FF
